:020000040800F2
:1000000000800020B3AB000815AB000829AC000845
:1000100019AB00081BAB00081DAB00080000000076
:100020000000000000000000000000001FAB0008FE
:1000300021AB00080000000023AB0008211E0008CF
:1000400027AB000829AB00082BAB00082DAB00083C
:100050002FAB000831AB000833AB000835AB00080C
:1000600037AB000839AB00083BAB00083DAB0008DC
:100070003FAB000841AB000843AB000845AB0008AC
:1000800047AB00080000000049AB00084BAB00087C
:10009000FD2D00084FAB000851AB000853AB000822
:1000A00055AB000857AB000859AB00085BAB000824
:1000B0005DAB00085FAB000861AB000863AB0008F4
:1000C00065AB000867AB000869AB00086BAB0008C4
:1000D0006DAB0008B91E000871AB000873AB0008D7
:1000E00075AB000877AB000879AB00087BAB000864
:1000F0007DAB00087FAB000881AB0008000000006A
:100100000000000083AB00080000000085AB000881
:1001100087AB00080000000089AB00088BAB00082B
:100120008DAB00088FAB000891AB000893AB0008C3
:1001300095AB0008000000000000000097AB00082D
:1001400099AB00089BAB0008000000000000000015
:10015000000000000000000000000000000000009F
:100160000000000000000000000000009DAB00083F
:100170009FAB00080000000000000000000000002D
:1001800000000000A1AB000800000000000000001B
:10019000000000000000000000000000000000005F
:1001A0000000000000000000A3AB0008A5AB0008A1
:1001B000A7AB0008A9AB0008ABAB0008000000002B
:1001C00000000000ADAB00080000000000000000CF
:0801D000AFAB0008B1AB000861
:1001D8002DE9F0411C4B1E683768384609F09AFF34
:1001E800044656F8048C404609F094FF214609F06D
:1001F80069FE09F0A7FF04460D460FA3D3E90023C3
:1002080009F036FF80B90EA3D3E90023204629461A
:1002180009F04AFF40B908FB07F746F8047C0A4A88
:100228001368043B136004E0084A136843F48063CE
:100238001360BDE8F08100BF0000C0FFFFFFDF4191
:100248000000C0FFFFFFDFC1B8760020FC76002069
:100258002DE9F047344B1C682568002D44D054F82C
:10026800088C54F8049C484609F054FF064640465A
:1002780009F050FF314609F025FE824609F062FF79
:1002880006460F4624A3D3E9002309F0F1FE38B946
:1002980023A3D3E900233046394609F005FF80B38C
:1002A800284609F037FF0146504609F071FE054619
:1002B80009F048FF06460F4617A3D3E9002309F0C3
:1002C800D7FEC0B916A3D3E900233046394609F052
:1002D800EBFE80B9A4F10802134B1A60284609F016
:1002E800FFFE44F8080C04E0104A136843F4006366
:1002F8001360BDE8F0870D4A136843F48063136008
:10030800F7E7A4F10802084B1A6009FB08F898FB04
:10031800F5F544F8085CECE70000C0FFFFFFDF419B
:100328000000C0FFFFFFDFC1B8760020FC76002088
:1003380008B5544B9A6D42F080529A651A6842F497
:1003480080321A6000234F490A68013312F4003FD3
:1003580015D1B3F5A02FF7D14A4A116821F480319D
:100368001160116841F48071116011460A68013307
:1003780012F4806F41D1B3F5A02FF7D33CE0424B84
:1003880040F202721A60A3F580539A689A609A68DC
:100398009A609A689A604FF44062DA60D3F88820CD
:1003A80022F04062C3F88820D3F8882042F0006227
:1003B800C3F88820DA6842F08872DA60DA6842F0B6
:1003C8000302DA601A6842F080721A601A461368EB
:1003D80013F0007FFBD02B4A936843F0030393602C
:1003E800936803F00C030C2BFAD102F043FF254A63
:1003F800936C43F48073936408BD234B40F20272FC
:100408001A60A3F580539A689A609A689A609A6805
:100418009A601022DA604FF44062DA60DA68DA60D3
:10042800DA68DA60D3F8882022F04062C3F88820BE
:10043800D3F8882042F00062C3F88820DA6842F0D6
:100448008872DA60DA6842F00202DA601A6842F00A
:1004580080721A601A46136813F0007FFBD0094AAD
:10046800936843F003039360936803F00C030C2B29
:10047800FAD102F0FFFE034A936C43F4807393644D
:0C048800BAE700BF001002400020024054
:100494004FF090434FF080729A61024B04221A602D
:0804A400704700BFA0770020A3
:1004AC00332303494AF6AA220A60013BFCD1704768
:0404BC0000300040CC
:1004C00010B506F061FB294AD2F80438DC43D2F8B3
:1004D0000818D2F8002813400B40B3F1FF3F38D082
:1004E000C843234B1C60234B1860204BD3F80C38B7
:1004F000DB4313F07F0232D01F490A601E4A1168A5
:100500001E4A1160C3F304431D4A13600A2B04D032
:10051000102B02D013460A221A60194B1A68194B85
:100520001A60124AD2F81038DB4317490B60D2F830
:100530001438DB43154A1360ABB10C4AD2F81838B3
:10054000DB4313490B60D2F81C38DB43114A1360BC
:1005500010BD0B23084A1360084A1360F8E7064AE7
:100560000B211160CAE706F00FFBE6E700B00008B8
:100570003877002094770020B07700208077002023
:10058000D876002080760020A87700209077002081
:080590002477002034770020DD
:100598002D4A136E43F4804313664FF0904213685C
:1005A80023F480131360136843F400131360274B7C
:1005B800196821F480511960196841F400511960D3
:1005C800516A21F470615162516A41F4E0615162EB
:1005D8001A6A22F070621A621A6A42F0E0621A62BB
:1005E8001B4B1C4A13601C4A13601C4B1B68262BB0
:1005F80021D008D9392B24D0602B14BF4FF4D072E6
:100608004FF49C5207E0132B18D01F2B14BF4FF444
:10061800D0724FF4C062124BDA604FF400325A6065
:1006280000229A602D221A600E4B01221A600E4B8E
:1006380020225A6070474FF49C62ECE74FF41C622A
:10064800E9E74FF45072E6E7001002400004004862
:10065800246300207C7700207877002080770020B2
:0C06680000380140AC77002000E100E009
:10067400034AD36913F0800FFBD0014B9862704793
:0406840000380140F9
:1006880010B504460C4B1B684BB1022B10D0042B41
:100698000ED00A4B1B6873B102F0B0FD0BE0FFF7F8
:1006A800E5FF064B1B6833B1204602F0A7FD02E0C8
:1006B8002046FFF7DBFF10BD887700205C7600201E
:1006C800F8B5864B1B68002B00F0E98003F5005352
:1006D80002339C032368B3F1FF3F33D00023804AE1
:1006E8001360804A13606368DB437F4A13600A2BF8
:1006F80004D0102B02D013460A221A607A4B1A68CB
:100708007A4B1A60A368DB43794A1360E368DB43DA
:10071800C3F30161774A1160C3F30541764A11605A
:100728009BB2764A13602269D243754B1A6063699B
:10073800DB43190C09D04FF6FF70814205D0714890
:10074800016006E006F01CFAA9E06E494FF0FF30A0
:1007580008609BB233B14FF6FF718B4202D06A49F1
:100768000B6003E0684B4FF0FF31196072B9A26962
:10077800D243664B1A60E369DB43190C0DD04FF680
:10078800FF70814209D0624801600AE006F0B8FCB7
:1007980006F030FD06F0B2FDE9E75D494FF0FF30A5
:1007A80008609BB233B14FF6FF718B4202D05949B2
:1007B8000B6003E0574B4FF0FF31196032B904F179
:1007C800300C554D05F5FC64AE4614E006F044FEC9
:1007D80006F0C6FE06F046FFF1E70B68DB43CEF8ED
:1007E80010304B68DB43CEF814300CF1180C0EF1C6
:1007F800180EA64510D0ACF11001724651F8043B12
:10080800DB431370180A5070180C90701B0ED370CD
:1008180004326145F2D1E0E7304B1C68013CA40387
:1008280004F1006606F54846DFF8F0C0A4443C4FE2
:1008380005F57C650AE00B68DB433B614B68DB43ED
:100848007B610CF1180C1837AF4210D0ACF11001D5
:100858003A4651F8043BDB431370180A5070180CE1
:1008680090701B0ED37004326145F2D1E3E7D6F8DD
:10087800E037DB432B4A1360D6F8E437DB432A4AD8
:1008880013602A4B03F54050C3F1006101F5504154
:10089800E2185258D24343F8042F9842F8D1FFF790
:1008A80001FE03F0F1FC124B1B6843B14FF090437B
:1008B8001B6913F4806F02D10D4B00221A600D20C2
:1008C800FFF7DEFE04F0A2FA094B1B6803B9F8BD76
:1008D800013B174A136008F0DDFBF8E7907700202A
:1008E8009C77002098770020D8760020807600201A
:1008F8001C770020A0760020A8760020A47600208F
:10090800F4760020D4760020D0760020F0760020FF
:10091800CC760020C8760020BC32002010C8000821
:100928009C3A00202477002034770020B802002069
:04093800C476002061
:10093C0008B5104B1B6823F00202012A09D0022BC8
:10094C000AD0042B0FD00C4A136843F080031360B9
:10095C0001E0FFF789FE08BD084B1B68002BF2D0A5
:10096C0002F04AFCF7E7054B1B68002BEBD002F0BA
:10097C0093FAF0E788770020FC7600205C76002064
:10098C0010B500F13004E4B2392C84BF3730C4B256
:10099C000E4B1B683BB123F00203012B0ED02046FB
:1009AC00FFF762FE10BD2046FFF75EFE084B1B688A
:1009BC00002BF7D0204602F01FFCF3E7044B1B681A
:1009CC00002BECD0204602F017FCEBE788770020D8
:0409DC005C76002025
:1009E0002DE9F0418CB007AC334D0FCD0FC42B680F
:1009F000236001AC314D0FCD0FC495E8030044F8DE
:100A0000040B24F8021B090C21702D4B01221A60E3
:100A10002C4B1B68042B14BF002301232A4A1360AC
:100A200001F096FB40F6B833284A1360DFF8A08047
:100A30004AF6AA271546274E07E02E20FFF724FE88
:100A40002346326872B92A6862B1C8F800702C680F
:100A50009C42F6D0C4F3090240F2FF339A42ECD034
:100A60002346EEE7174B1B68042B0CBF01A807A811
:100A70000AF011FC174B1B6873B16F20FFF704FEDF
:100A80006B20FFF701FE0D20FFF7FEFDC82000F0F0
:100A9000EBF80CB0BDE8F0816520FFF7F5FD7220A2
:100AA000FFF7F2FD7220FFF7EFFD6F20FFF7ECFD7F
:100AB0007220FFF7E9FDE6E7CCAF0008E0AF0008E1
:100AC0003C7700208877002058760020847700202B
:080AD000003000405C760020BC
:100AD80010B58AB00DF1140C514C0FCCACE80F00D6
:100AE80023688CF800304F4B01AC0FCB07C4238030
:100AF8004D4BDB6913F0800F0BD04C4A13684C49FF
:100B0800C85C49498862013313604A4A12689342B3
:100B180015D2494B1B6883B9474B0A221A60474BC9
:100B28004AF6AA221A60464B1B685BB9454B1B68FC
:100B38005A1C042B09D0434B1A600AB010BD09F0A7
:100B4800F9F8E6E709F06EF9F0E73E4B00221A6083
:100B58003D4B1B685BB1013B3B4A13603BB13B4BD0
:100B68001B685A1C132B08D0384B1A60E5E74FF066
:100B780090434FF480729A61F1E7344B00221A6077
:100B8800334B1B6893B94FF090431B6913F4007FF4
:100B9800D3D0304B1B68002BCFD105A80AF077FBC8
:100BA8000D20FFF76DFDFFF717FFC6E74FF09043E5
:100BB8001B6913F4007F17D0274B1B68042B1FD029
:100BC800254B1B68032BB8D8244B1B68012BB4D1C9
:100BD80001F0B0F9214B00221A604FF4FA7000F0CE
:100BE8003FF8FFF7F9FEA8E701A80AF050FB0D202F
:100BF800FFF746FD01F09EF9164B00221A609CE7AC
:100C0800164B1B68002B98D101F094F9134B012265
:100C18001A604FF4FA7000F023F8FFF7DDFECFE713
:100C280040AC000854AC000800440040287700207D
:100C38003C6F00202C7700208C770020003000408B
:100C480020770020B8770020A07700203876002091
:100C58005C7600203C7700208877002058760020BA
:100C6800054B186038B110B51C46FFF731FF2368F3
:0C0C7800002BFAD110BD7047A4770020BB
:100C840008B5574B186910F48030FBD1544B5B699D
:100C9400002B80F29580524B524A9A6002F18832BE
:100CA4009A60A3F5F8334AF6AA221A604C4A1369EB
:100CB40013F4803FFBD14A4B4B4A5A615A6942F4C0
:100CC40080325A61186910F48030FBD1444B1A69A0
:100CD40042F001021A611B6913F0020F70D1404BFC
:100CE4005A6922F002025A615A6942F001025A61B9
:100CF4003E4A0023C2F800383D4B1B88DB43C2F850
:100D04000438374B186910F48030FBD1344B1A691E
:100D140042F001021A611B6913F0020F50D1334AE9
:100D2400344B1B88DB43C2F80838334B1B6803F091
:100D34007F033249096843EA0143DB43C2F80C38B4
:100D4400274B186910F48030FBD1254B1A6942F007
:100D540001021A611B6913F0020F31D1234A284B97
:100D64001B68DB43C2F81038264B1B68DB43C2F810
:100D740014381B4B186910F48030FBD1184B1A69D6
:100D840042F001021A611B6913F0020F18D1174ACD
:100D94001D4B1B68DB43C2F818381C4B1B68DB4334
:100DA400C2F81C380E4B186910F48030FBD10C4B80
:100DB4001A6942F001021A611B6913F0020F00D094
:100DC40008BD074B5A6922F001025A615A6942F080
:100DD40000425A611420FFF745FF0120F0E700BFED
:100DE4000020024023016745BA00000300B0000858
:100DF4003877002094770020B0770020D876002040
:100E0400A8770020907700202477002034770020F2
:100E1400904B1B68002B00F06D842DE9F0478CB0DB
:100E24008D4A136913F4803FFBD18B4B5B69002B14
:100E3400C0F2A980894B4AF6AA221A60854B1C6825
:100E4400013CE400844A136913F4803FFBD104F1AC
:100E54001803DB0043F0407343F002037E4A5361FE
:100E6400536943F4803353611346186910F4803096
:100E7400FBD1794B1A6942F001021A611B6913F024
:100E8400020F40F01184744B5A6922F002025A6135
:100E940004F580321832D202596941F001015961D6
:100EA400002313606E4B1B68DB4353606A4B186965
:100EB40010F48030FBD1684B196941F001011961CC
:100EC4001B6913F0020F40F0EF83664B1B68DB4392
:100ED4009360654B1968654B1B681B0443EA016307
:100EE400634909680B43DB43D3605B4B186910F417
:100EF4008030FBD1584B196941F0010119611B691C
:100F040013F0020F40F0D0835A4B1B68DB4313618C
:100F1400594B1968594B1B8843EA0143DB4353611E
:100F24004D4B186910F48030FBD14B4B196941F0DB
:100F3400010119611B6913F0020F40F0B583504B96
:100F44001B68DB4393614F4B19684F4B1B8843EA83
:100F54000143DB43D361404B186910F48030FBD16B
:100F64003D4B196941F0010119611B6913F0020F2E
:100F740040F09A832032454F07F5FC6EBC4604AE20
:100F84000AAD354B0AE0344B414A9A6002F188328B
:100F94009A604FE70CF1300CF4457BD0E84660468C
:100FA40090F801908178090441EA092190F80090B1
:100FB40041EA090190F8039041EA096148F8041BE9
:100FC4000430B045ECD16046DCF810100491DCF834
:100FD400141005910DF11809E04698F819A098F835
:100FE4001A10090441EA0A2198F818A041EA0A01F2
:100FF40098F81BA041EA0A6149F8041B08F10408A7
:10100400A945EAD1816A0A91C16A0B9102F10808E3
:1010140002F1380AE9464246D9F80010C94348F8B3
:10102400081CD9F80410C94348F8041C186910F4C2
:101034008030FBD1196941F001011961196911F07E
:10104400020F40F0318308F1080809F10809D0457E
:10105400E1D19FE79077002000200240003000405B
:10106400D87600201C770020A0760020A8760020E7
:10107400A4760020F4760020D4760020D0760020D8
:10108400F0760020CC760020C8760020BC32002008
:1010940023016745564A536923F001035361554BB5
:1010A4004AF6AA221A602E20FFF7ECFA504A136976
:1010B40013F4803FFBD14E4B5B69002B35DB4C4A6C
:1010C400136913F4803FFBD104F11903DB0043F0EF
:1010D400407343F00203464A5361536943F4803337
:1010E40053611346186910F48030FBD1404B1A69E0
:1010F40042F001021A611B6913F0020F40F0D4821E
:101104003B4B5A6922F002025A6104F5803808F117
:1011140019084FEAC8284246596941F0010159614A
:10112400DFF8D4C007F57C670AE0314B334A9A6094
:1011340002F188329A60C2E70CF1300CBC455FD0F2
:10114400EE46604690F801908178090441EA09214D
:1011540090F8009041EA090190F8039041EA09618E
:101164004EF8041B0430B645ECD16046DCF8101090
:101174000491DCF8141005910DF11809E6469EF867
:1011840019A09EF81A10090441EA0A219EF818A031
:1011940041EA0A019EF81BA041EA0A6149F8041BCE
:1011A4000EF1040EA945EAD1816A0A91C16A0B9134
:1011B40002F13009EE46DEF80010C9431160DEF892
:1011C4000410C943516092460832186910F4803003
:1011D400FBD1196941F001011961196911F0020F7C
:1011E40040F062820EF1080E4A45E4D1A4E700BF44
:1011F40000200240003000409C3A00202301674553
:10120400A94B1B68DB43CAF80830A84B1B68DB43B7
:10121400CAF80C30A64B186910F48030FBD1A44BEB
:101224001A6942F001021A611B6913F0020F40F0BF
:101234003B829F4A536923F0010353619D4B4AF655
:10124400AA221A6003F5F8331A6912F4803FFBD11D
:10125400974B5B69002BC0F22A82954B1A6912F4F2
:10126400803FFBD104F11A03DB0043F0407343F0E9
:1012740002038F4A5361536943F480335361134625
:10128400186910F48030FBD1894B1A6942F00102CD
:101294001A611B6913F0020F40F00682844A5369F5
:1012A40023F00203536108F50063516941F0010121
:1012B400516108F580558049A1EB08010F1DC858FC
:1012C400C0431860F858C04358600833106910F4DC
:1012D4008030FBD1166946F001061661166916F0D6
:1012E400020F40F0E1819D42E9D1714A536923F034
:1012F400010353616F4B4AF6AA221A602E20FFF7AE
:10130400C1F96B4B1A6912F4803FFBD1684B5B69DE
:10131400002BC0F2D381664B1A6912F4803FFBD1D3
:1013240004F11B03DB0043F0407343F00203604A03
:101334005361536943F4803353611346186910F4BD
:101344008030FBD15A4B1A6942F001021A611B69C1
:1013540013F0020F40F0A881554B5A6922F00202A3
:101364005A615A6942F001025A61544908F5C0525F
:10137400D1F80008C0432860D1F80408C04368606D
:101384000835186910F48030FBD11E6946F0010657
:101394001E611E6916F0020F40F086810831AA42D0
:1013A400E6D143494B6923F001034B61414B4AF6B3
:1013B400AA21196003F5F833196911F4803FFBD1B0
:1013C4003B4B5B69002BC0F28081394B196911F4E6
:1013D400803FFBD104F11C03DB0043F0407343F076
:1013E400020333494B614B6943F480334B610B4631
:1013F400186910F48030FBD12D4B196941F00101BB
:1014040019611B6913F0020F40F04E81284B596992
:1014140021F002015961596941F0010159612849DA
:1014240008F500550868C04310604868C043506020
:101434000832186910F48030FBD11E6946F00106A9
:101444001E611E6916F0020F40F02E81083195428C
:10145400E8D1174A536923F001035361154B4AF647
:10146400AA221A602E20FFF70DF9114B1A6912F403
:10147400803FFBD10E4B5B69002BC0F22D810C4BDE
:101484001A6912F4803FFBD104F11D03DB0043F021
:10149400407343F00203064A5361536943F48033B3
:1014A400536113460EE000BF2477002034770020F8
:1014B4000020024000300040BCFAFF1FBC020020A4
:1014C400BC120020186910F48030FBD18A4B1A69D1
:1014D40042F001021A611B6913F0020F40F0E4802C
:1014E400854B5A6922F002025A615A6942F001029C
:1014F4005A61824908F520520868C0432860486848
:10150400C04368600835186910F48030FBD11E6947
:1015140046F001061E611E6916F0020F40F0C480F9
:1015240008319542E8D174494B6923F001034B61BA
:10153400734B4AF6AA21196003F5F833196911F4BB
:10154400803FFBD16C4B5B69002BC0F2CC806A4BB3
:10155400196911F4803FFBD104F11E03DB0043F051
:10156400407343F0020364494B614B6943F4803395
:101574004B610B46186910F48030FBD15E4B19693E
:1015840041F0010119611B6913F0020F40F08C80D6
:10159400594B596921F002015961596941F001011E
:1015A4005961584908F540550868C04310604868B7
:1015B400C04350600832186910F48030FBD11E69B2
:1015C40046F001061E611E6916F0020F6CD1083147
:1015D400AA42E9D1484A536923F001035361484BB5
:1015E4004AF6AA221A602E20FFF74CF8424B1A69D9
:1015F40012F4803FFBD1404B5B69002B05DA3E4B74
:10160400414A9A6002F188329A603B4B1A6912F49B
:10161400803FFBD104F11F03DB0043F0407343F030
:101624000203354A5361536943F4803353611346CB
:10163400186910F48030FBD12F4B1A6942F0010273
:101644001A611B6913F0020F2ED12B4B5A6922F039
:1016540002025A615A6942F001025A612B4A08F5A2
:1016640060581168C94329605168C94369600835E5
:10167400186910F48030FBD1196941F00101196136
:10168400196911F0020F0FD10832A845E9D11A4B9C
:101694005A6922F001025A615A6942F000425A61C1
:1016A4001420FFF7DFFA01200CB0BDE8F087124BDD
:1016B400154A9A6002F188329A60CEE50E4B124ABE
:1016C4009A6002F188329A6025E60B4B0E499960C4
:1016D40001F18831996078E6074B0B4A9A6002F170
:1016E40088329A60CBE6044B0749996001F188314E
:1016F40099602CE70120704700200240BC1A0020AA
:1017040000300040BC22002023016745BC2A002091
:1017140010B50446384A136913F4803FFBD1364BA5
:101724005B69002B61DB354B4AF6AA221A602E2036
:10173400FEF7A8FF304A136913F4803FFBD104F18C
:101744002803DB0043F0407343F002032A4A536149
:10175400536943F4803353611346186910F480309D
:10176400FBD1254B1A6942F001021A611B6913F07F
:10177400020F39D1204B5A6922F002025A615A6988
:1017840042F001025A6104F5803428341C4AC2EB49
:10179400C42C194B02F500640CEB02001168C94318
:1017A4004CF802105168C94341600832186910F4BA
:1017B4008030FBD1196941F001011961196911F0F7
:1017C400020F11D1A242E7D10B4C636923F001034C
:1017D40063612E20FEF756FF636943F000436361A3
:1017E4000A20FFF73FFA012010BD034B054A9A6017
:1017F40002F188329A6096E70020024000300040EF
:081804001C520020230167457E
:10180C0010B5041E7ADB092C72D9632C64D9B4F59B
:10181C007A7F56D342F20F739C4246D9404B9C427E
:10182C0037D9404B9C4228D93F4B9C421AD33F4B53
:10183C009C420CD93E4B9C4265D83E48A0FB0430E0
:10184C00400E3D4B03FB10443030FEF717FF3B4876
:10185C00A0FB0430800D344B03FB10443030C0B27D
:10186C00FEF70CFF3648A0FB0430800C354B03FB15
:10187C0010443030C0B2FEF701FF6009324BA3FBBD
:10188C000030C009314B03FB10443030C0B2FEF7BE
:10189C00F5FE2F48A0FB0430400B42F2107303FB03
:1018AC0010443030C0B2FEF7E9FE2A48A0FB0430E9
:1018BC0080094FF47A7303FB10443030C0B2FEF74A
:1018CC00DDFE2548A0FB04304009642303FB1044D3
:1018DC003030C0B2FEF7D2FE2048A0FB0430C00866
:1018EC0000EB8003A4EB43043030C0B2FEF7C6FE1D
:1018FC0004F13000C0B2FEF7C1FE10BD2D20FEF782
:10190C00BDFE64427FE7600A154BA3FB0030C009A3
:10191C00144B03FB10443030FEF7B0FE8DE700BFD4
:10192C009F8601003F420F0080969800FFE0F5056E
:10193C00FFC99A3B893BE65500E1F5056BCA5F6B25
:10194C0083DE1B4340420F00C55A7C0AA08601006F
:10195C005917B7D1D34D62101F85EB51CDCCCCCCE0
:08196C00834B040000CA9A3B02
:1019740030B591B00DF11C0C144C0FCCACE80F0039
:101984000FCCACE80F002368ACF800306C46104D67
:101994000FCD0FC495E8070003C422700D20FEF795
:1019A40071FE07A809F075FC3720FEF76BFE2E20A8
:1019B400FEF768FE3D20FFF727FF684609F069FC43
:1019C4000D20FEF75FFE11B030BD00BFF8AF000878
:0419D4001CB000083B
:1019D80008B508F03BF908F0ADF90220FFF740F927
:1019E8000D20FEF74DFEFFF7C1FF0C4B00221A60D9
:1019F8004FF090431B6913F4007F05D0084B1B6818
:101A080013B1084B1B6833B9074809F040FC0D2097
:101A1800FEF736FE08BDFEF7DFFFFBE75C76002029
:0C1A2800387700209477002038B00008C8
:101A340008B5594B9A6D42F080529A65DA6C42F0BF
:101A44000102DA64DA6C42F00202DA644FF0904583
:101A540000242C60514B1C60514AEA604FF0AA32BA
:101A6400DA60FEF767FCEB6823F44033EB602B6825
:101A740023F440332B602B6843F480332B604FF402
:101A84008073AB61EB6823F44023EB60454B142275
:101A94001A60454B1C60454B1C60454B1C60454B14
:101AA40040F283421A60444B45F240721A60434B41
:101AB4001C60434B1C60434B1C60434B434A1A60FD
:101AC4000A23434A1360434A1360434B1C600B23AD
:101AD400424A1360424A1360424B1C60424B1C60F2
:101AE400424B1C60424B1C60424B4FF400721A6024
:101AF400414B1B68414AA2FB03239B09013BB3F101
:101B0400807F09D24FF0E02253613D4BF02183F8EE
:101B140023109461072313613220FFF7A3F8394C93
:101B240045F2555323604FF6FF73A3600220FFF77D
:101B340099F8022565602846FFF794F84CF6CC43E3
:101B44002360FEF7BBFC2846FFF78CF8FEF722FD66
:101B54000520FFF787F8FFF73DFFFEF7B3FD2A4B9B
:101B64001B6863B9294CFEF7B5FF04F07BF806F057
:101B740081FE2368002BF6D007F0FEFAF3E702F0AB
:101B840063FB234A1368191D11601F4A12685A60C7
:101B940003F084FFE6E700BF0010024000040048A1
:101BA400AAAA02A88C770020A0770020A47700209E
:101BB400847700203877002094770020587600201E
:101BC4003C77002090770020BC760020A1B0B912A9
:101BD400D87600208076002088770020B077002017
:101BE40080770020AC770020A87700209C77002025
:101BF400987700202C770020B8020020D34D621083
:101C040000ED00E0003000403477002074760020BE
:041C1400B87600207E
:101C180010B5FEF75DFF0C4B1B680C4A1268934227
:101C280010D05A1C08490A601C7844F40044084B38
:101C38001B689A4203D0FEF729FC204610BD054ACE
:101C48000A60F8E70024F8E7787700207C7700201E
:081C5800B40200202463002007
:101C600008B50D4B1B6843B90C4B1B6813B100F052
:101C7000EFFE08B9FFF7D0FF08BD022B08D0042BF8
:101C800006D0064B1B68002BF6D000F0E1FEF3E710
:101C9000FFF7C2FFF0E700BF887700205C760020E6
:101CA0007F2845D9A0F1F0030D2B06D842F2B122CE
:101CB00022FA03F313F0010F16D1F6281CD0F728EF
:101CC0001AD8414B1A6800F00F03511E8B4201D005
:101CD000002A25D13D4B186000F0F0003C4B186005
:101CE0003C4B01221A60704700233A4A1360374A7E
:101CF0001360374A13607047374B1B680004374A3C
:101D000042F823005A1C7F2B334B08BF00221A6075
:101D10000023304A13602D4A13602D4A1360704728
:101D200000232C4A1360294A1360294A1360704724
:101D3000284B1B6823B1012B09D0022B29D07047F7
:101D4000224A1360224A1360254A13607047244BCD
:101D500018601F4B1B6823F01003C02B09D01B4BCE
:101D60001B6823F00203F12B03D01A4B02221A60E6
:101D70007047194B1B68154A126840EA0240174A1F
:101D800042F823005A1C7F2B134B08BF00221A6015
:101D90007047114B1A680D4B1968114B1B681B02D9
:101DA00043EA014318430D4B43F82200531C7F2A9A
:101DB00005D0094A1360074B01221A60BFE7064BA2
:101DC00000221A60F7E700BFA877002034760020D1
:101DD000407600203C7600209C7700204071002057
:041DE000B4770020B4
:101DE40008B5FEF777FE0A4B1B680A4A126893424D
:101DF4000BD0094A52F8230040F000405A1C7F2BB4
:101E0400034B08BF00221A6008BD0020FCE700BF96
:0C1E1400987700209C770020407100208F
:101E20001C4B1B6813B1013B1A4A13601A4B1B6809
:101E300013B1013B184A1360184B1B6813B1013BE7
:101E4000164A1360164B1B6813B1013B144A13600A
:101E5000144B1B6813B1013B124A1360124B1B68F1
:101E600013B1013B104A1360104B1B6813B1013BC7
:101E70000E4A13600E4B1B6813B1013B0C4A1360F2
:101E80000C4A136883EA433383EA534383EA4313D8
:101E9000136070478C770020A4770020847700209F
:101EA000E476002084760020B4760020B07600200E
:081EB000AC760020BC76002096
:101EB80008B51A4BDB6913F0200F2AD0174B5A6A62
:101EC800174B1B6823F00203012B18D0D3B2022B47
:101ED8000ED0042B10D013490B681A700B6801330D
:101EE8000B60114A1268934213D1104A0A6010E03D
:101EF8000F4B02211960EEE702F04CFC09E009499A
:101F08000B681A700B6801330B60074A126893421A
:101F180000D008BD054A0A60FBE700BF0038014051
:101F2800887700207C770020B402002024630020FA
:041F38007876002097
:101F3C004FF090431A6A22F07F421A621A6822F01C
:101F4C0070721A60144B4FF40022C3F88020BFF358
:101F5C004F8FBFF36F8F4FF48012C3F88020BFF305
:101F6C004F8FBFF36F8F02F18042A2F55F22936B0C
:101F7C0043F4000393630949B1F840309BB243F03A
:101F8C000203A1F84030936D23F400039365044BD6
:101F9C0000221A60704700BF00E100E0005C0040C6
:041FAC005C7600203F
:101FB0004F4A8023A2F84C3000214E4B1960B2F8F2
:101FC00058306FEA43436FEA53439BB2A2F858304C
:101FD000A2F85010B2F850309BB203F1804303F5E1
:101FE000C043454A1360454A1360991C444A116036
:101FF000191D444A1160991D434A116003F10801FB
:10200000424A116003F10A01414A116003F11401CF
:10201000404A116003F116013F4A11603F4A1268BD
:102020003AB903F118023E490A6003F11A023D4928
:102030000A6040221A80324B1B6800221A80314B02
:102040001B6880211980304B1B684FF404411980B4
:102050002E4B1B684FF4807018802D4B1B681A8024
:10206000254B1B689881DA814FF4007018825A82E0
:10207000284B1B681880284B1B681980274B1B684E
:102080005BB9274B1B684FF440711980254B1B68C7
:102090001A80194B1B689983DA83154B43F220226F
:1020A0001A8043F231029A8043F232021A811B4BAA
:1020B0001B681BB90E4B43F233629A810C4B4FF4F1
:1020C0003F42A3F840200023174A1360174A1360C9
:1020D000174A18490A6018490A60184A18490A60DC
:1020E00018490A60184A1370184A1370704700BFE5
:1020F000005C00406476002060760020707700204D
:102100005C77002074770020607700206C770020D7
:1021100058770020687700205477002058760020F8
:102120006477002050770020447600205C76002001
:102130001C5A00204477002040770020A05E002039
:102140004C7700204877002029670020316B002061
:1021500010B5234CA36D43F40003A365A36B43F4B4
:102160000003A363FEF7A2F9A36B23F40003A363A8
:102170004FF090431A6822F070721A60DA6822F009
:102180007072DA60174B00221A60174B1146174A1B
:1021900023F8021B9342FBD1154B0021154A23F86B
:1021A000021B9342FBD1104CB4F858306FEA434302
:1021B0006FEA53439BB2A4F858300123A4F840308F
:1021C000C820FEF751FD0023A4F84030A4F84430A5
:1021D000FFF7EEFE084B4FF480121A6010BD00BFEF
:1021E0000010024048760020005C0040205C004067
:0C21F000445C0040605C004000E100E046
:1021FC0070B483B0304B1B68402B55D92F4B1B68E8
:10220C0040221A802C4A1368403B13602B4B1B68EE
:10221C001B88BBB12A4D00222A4C284E2368184635
:10222C0010F8011B206058780233236041EA002328
:10223C0025F8023B013292B233681B880133B2EBB2
:10224C00630FEBDB204B1B8813F0800F08D01E4A6A
:10225C0013889BB223F4E14323F070039BB21380E9
:10226C001A4B1B684FF404421A80174B1B889BB205
:10227C00ADF80630BDF8063013F0200F03D1124B29
:10228C0048F2A0221A80104B1B889BB2ADF8063086
:10229C00BDF8063013F0100F03D10B4B48F290220F
:1022AC001A8003B070BC7047034B1968034A12685C
:1022BC00118000221A60A9E7447600205C77002088
:1022CC004060004050760020005C004060770020A9
:1022DC0082B01B4B1B6800221A801A4B1B889BB2C6
:1022EC00ADF80630BDF8063013F0800F09D0BDF8FC
:1022FC0006309BB223F4E14323F070039BB2114AE6
:10230C001380104B1B889BB2ADF80630BDF806301D
:10231C0013F0200F03D10B4B48F2A0221A80094B6B
:10232C001B889BB2ADF80630BDF8063013F0100FC9
:10233C0003D1044B48F290221A8002B0704700BFC0
:08234C005C770020005C0040FA
:1023540000B583B0274A13889BB223F4E14323F0EA
:1023640070039BB21380244B1B68052B2BD0234B8B
:102374001B68002B3AD11F4B1B8813F4004F2DD13F
:102384001C4B1B889BB2ADF80630BDF8063013F425
:10239400005F03D1174B4AF280221A80154B1B8829
:1023A4009BB2ADF80630BDF8063013F4805F03D15C
:1023B400104B49F280221A80114B1B6800221A80AC
:1023C40003B05DF804FB0F4B1B6843F080039BB222
:1023D400A2F84C30084B00221A60C8E7054A13885B
:1023E40023F070031B051B0D1380C9E7FFF704FFDF
:1023F400E6E700BF005C00404876002044760020F9
:082404005C77002064760020E3
:10240C0082B01F4B1A8822F070021205120D1A802E
:10241C001B8813F0800F08D0194A13889BB223F441
:10242C00E14323F070039BB21380154B1B889BB2C6
:10243C00ADF80630BDF8063013F0100F03D1104B79
:10244C0048F290221A800E4A13889BB2ADF80630DF
:10245C00BDF8063013889BB2ADF80630BDF80630D7
:10246C0013F4805F03D1134649F280221A80044B87
:10247C001B889BB2ADF80630BDF8063002B0704731
:04248C00005C0040B0
:1024900030B587B0924B1B8813F4006F00F0E581D4
:1024A000904B93F880209048027093F881108F4AE7
:1024B0001170B3F882108E4A11801188C1F3072180
:1024C0008C4C21701288D2B28B490A70B3F88410F8
:1024D0008A4A1180B3F88620894B1A80894B0022E2
:1024E0001A60894B1B684FF404421A800378DBB2F0
:1024F000212B29D07C4B1B78DBB2A12B7ED07A4BD1
:102500001B7813F0610F06D0774B1B7803F0610343
:10251000012B40F0A781724A138823F070031B053A
:102520001B0D1380714B1B78DBB2092B00F28A81E3
:10253000DFE813F08A008801880188018801930090
:10254000A200880188017F01704B1B68002BD1D14C
:10255000664B1B78DBB2202B0ED0644B1B78DBB2B2
:10256000222B48D15E4A138823F070031B051B0DF4
:102570001380FFF7B3FE84E1594B1B889BB2ADF883
:102580001630BDF8163013F4005F03D1544B4AF2F5
:1025900080221A80FDF78AFF514B1B889BB2ADF851
:1025A0001630BDF8163013F4805F03D14C4B49F25E
:1025B00080221A80FDF77AFF494B1B889BB2ADF849
:1025C0001630BDF8163013F4804F03D0444B4FF44F
:1025D00020721A80FDF76AFF414B1B8813F4004FED
:1025E00006D03F4CFDF762FF238813F4004FF9D16A
:1025F000FDF75CFF45E1FFF709FF42E13B4B1B782C
:10260000DBB2212B7FF47BAF404B1B68002B7FF4A8
:1026100076AF334A138823F070031B051B0D13801C
:102620003B4A07231360364B1B889BB212689342C8
:1026300004D2334B1B889BB2354A1360354B364A64
:102640001A60FFF7DBFD1CE1314B02221A60314BAF
:10265000324A1A60FFF7D2FD13E12D4B00221A60B7
:10266000FFF73CFE224B1B8803F07F032C4A1360CC
:10267000244B05221A6004E11E4B1B78DBB2012BB0
:1026800052D01C4B1B78DBB2022B00F08A80194B16
:102690001B78DBB2032B40F0C980174B1B78DBB2F1
:1026A000012B00F09C80144B1B78DBB2022B00F056
:1026B000A880114B1B78002B40F0B580144A0423EE
:1026C00013600F4B1B889BB21268934204D20C4BD1
:1026D0001B889BB20E4A13600E4B124A1A6056E0DA
:1026E000005C004000600040356D0020366D002029
:1026F0002A670020BC770020BD770020326B0020C5
:102700002E6900204876002060770020587600204F
:10271000447600205076002084B00008CCAC00083D
:102720006476002080A100085B4B12221A605B4B8C
:102730001A685B4C5B4B012A18BF1C465A4B1C6045
:102740005A4B1D6840F283439D4223D0621E01AB69
:102750000DF1160012F8011F03F8011B9842F9D180
:102760008DF80C502D0A8DF80D504D4B9C42504B5E
:1027700003BF1B680333DBB21B788DF80E304C4B64
:102780001B681B0A8DF80F30474B01AA1A60FFF730
:1027900035FD76E0464B1A6845F240739A42D5D132
:1027A000F5E73E4B1B68012B12D03B4B43221A60CE
:1027B0003D4B404A1A60404B1B889BB2364A126818
:1027C0009342E4D23C4B1B889BB2334A1360DEE752
:1027D000314B65221A60344B384A1A60EBE72E4AB7
:1027E00018231360344B1B889BB21268934204D2A7
:1027F000314B1B889BB2284A13602B4B304A1A601E
:10280000C5E7254A122313602B4B1B889BB2126825
:10281000934204D2284B1B889BB21F4A1360224B61
:10282000284A1A60B3E7FFF7F1FD2AE0FFF7EEFD53
:1028300027E0194B00221A60FFF750FD224BFF22C0
:102840001A601EE0214B1B7813B1FFF7DFFD18E083
:102850001F4A138823F070031B051B0D1380FFF71D
:102860003DFD0EE0FFF7D2FD0BE0194B1B889BB23C
:10287000ADF81630BDF8163013F4004F03D1FFF752
:102880002DFD07B030BDBDF8163023F070031B05D9
:102890001B0D0F4A1380F2E7447600205876002083
:1028A000FCAC0008ACAC0008507600203877002063
:1028B0009477002040B000082E6900208CB00008FA
:1028C00084A10008E0AC00085C760020356D002093
:0428D000005C004068
:1028D4002DE9F04383B03B4B9B8813F0800F08D065
:1028E400384A93889BB223F4E14323F070039BB2EC
:1028F4009380354800223549354D9646354E364C41
:102904002DE0BDF80430ACF800304A46334B1B6868
:102914001A802C4B9B889BB2ADF80630BDF806306C
:1029240013F0200F03D1274B48F2A1029A80BDF87F
:10293400063013F0100F03D1224B48F291029A8013
:1029440003B0BDE8F083BDF802309AB2BDF804309C
:102954009BB243EA0223ACF800304A460230A0F1AD
:10296400020C0B68D5F800804345CFD0ADF802E0E7
:1029740013F8017BADF804703768BB4208BF2346E7
:102984000B6002F101095FFA89F9B9F1400FB8D07F
:102994000B684345D7D013F8018BADF802809F42F2
:1029A40008BF23460B600232D2B2BDF802309FB298
:1029B400BDF804309BB243EA0723ACF80030402A48
:1029C400CCD1A3E7005C00400261004040770020C6
:1029D40044770020AC0200201C5A002058770020C5
:1029E40082B0184B9B8913F0800F08D0154A938945
:1029F4009BB223F4E14323F070039BB29381124B07
:102A04001B6800221A800F4B9B899BB2ADF80630DD
:102A1400BDF8063013F0200F03D10A4B48F2A3622D
:102A24009A81084B9B899BB2ADF80630BDF80630FD
:102A340013F0100F03D1034B48F293629A8102B052
:0C2A4400704700BF005C0040507700208D
:102A500010B5FEF741F8204B1868002834D01F4B02
:102A60001A681F4B1B689A4233D0511C1B480160E7
:102A70001078C4B21B4A1268914226D0174A1268D5
:102A8000934238BF03F590639B1A174A1268BAB194
:102A900040F23942934213D8134B00221A60134B71
:102AA0001B899AB213F4005F03D1104B4AF28201E2
:102AB000198112F4805F03D10C4B49F282021A8112
:102AC000FDF7E8FC44F4004010BD044A08491160D9
:102AD000D4E70020F8E700BF5C76002048770020AC
:102AE0004C770020B00200204C760020005C0040B3
:042AF000A05E0020C4
:102AF4006B4B19684A1C1A60012800F0CB8010B592
:102B04000B4613F8022B664C2360022800F0C480A5
:102B140091F801C0CB1C2360032800F0BF8091F81A
:102B240002E00B1D23600438C0B2931EDBB20D2BF0
:102B340000F2B380052A36D00F2A34D0A2F10C0358
:102B4400DBB2012B41D902F0FB03022B62D0C9781E
:102B5400072A00F28480534B00221A70524B1A68E1
:102B6400541C1C6082F800C01A68504B1B689A42BF
:102B740071D04D4B1A68541C1C6082F800E01A682E
:102B84004A4B1B689A4200F08180474B1A68541CD8
:102B94001C6011701A68454B1B689A427DD1424BE8
:102BA400434A1A6079E03F4B00221A703E4B1A6880
:102BB400511C196082F800C01A683C4B1B689A4289
:102BC4006BD1394B3A4A1A6067E0364B1B78634540
:102BD4000DD0354B1A68511C196082F800C01A6870
:102BE400324B1B689A4211D02E4B83F800C02E4BF7
:102BF4001A68511C196082F800E01A682B4B1B6894
:102C04009A424AD1284B2A4A1A6046E0264B284A5F
:102C14001A60E9E7234B00221A70234B1A68511CEF
:102C2400196082F800C01A68204B1B689A420ED0C3
:102C34001D4B1A68511C196082F800E01A681B4B7E
:102C44001B689A4229D1184B194A1A6025E0164B81
:102C5400174A1A60ECE7144B154A1A6089E7114BBE
:102C64001B78634585D0104B1A68541C1C6082F88D
:102C740000C01A680D4B1B689A4203D0094B83F8B5
:102C840000C076E7084B0A4A1A60F7E7064B084A81
:102C94001A607AE700207047002010BD0020FCE78E
:102CA40054760020316B00204C770020B0020020C5
:042CB400A05E0020FE
:102CB80070B582B0434B1B8913F4004F11D1424BBE
:102CC800424A1A60424B1B681878424B1B6803EB58
:102CD800430290423DD940283BD83F4E3A4C3F4DA5
:102CE80028E0384A138923F070031B051B0D138154
:102CF800E5E7FFF7FBFE15E0394B02221A600CE00E
:102D080022682B68591C296012781A702A68354B7A
:102D18001B689A4204BF344B2B602368013323603D
:102D28000138C0B22B4B1B6803EB4302904210D909
:102D380040280ED8012BDCD03368022BE0D0236862
:102D48001B78022BD8D0042BDAD1254B04221A6029
:102D5800E3E7264B1A68214B1B689A42A3EB020350
:102D680088BF03F590639BB2ADF80430204B002276
:102D78001A60BDF804309BB240F23A4293421CD824
:102D8800104B1B899BB2ADF80630BDF8063013F422
:102D9800005F03D10B4B4AF282021A81094B1B894F
:102DA8009BB2ADF80630BDF8063013F4805F07D14A
:102DB800044B49F282021A8102E00D4BFF221A608D
:102DC80002B070BD005C00405476002000620040F4
:102DD8005477002058760020887700204C77002010
:102DE80078760020B0020020A05E002048770020FE
:042DF8004C760020F5
:102DFC0000B585B0264BB3F844309BB20193019BD0
:102E0C0013F4004F26D0019B03F00F030393019B97
:102E1C0003F010030293039B012B09D0039B022B9D
:102E2C0009D0039B6BB9029B43B9FFF78DFA24E0E1
:102E3C00FFF74AFD21E0FFF739FF1EE0FFF722FB09
:102E4C001BE0039B032B18D1124B1B68ABB9FFF78C
:102E5C00C3FD12E00E4BB3F8443013F4806F0FD166
:102E6C000B4BB3F8443013F4006F094B14BF4FF203
:102E7C00FF7248F27F02A3F8442005B05DF804FB12
:102E8C00FFF790F8024B4FF6FF32A3F84420F4E71B
:082E9C00005C004058760020A4
:102EA400834A13780133DBB2137010F0800F20D102
:102EB400804B1B78002B00F09F807F4B1B7803F026
:102EC400F0017E4A1278002A40F0B9807C4A1070E2
:102ED4007C4A0020107003F0FD02F12A00F0958076
:102EE40003F0E003C02B00F09C80744BFF221A70A7
:102EF4007047F72800F04881134601221A70F02821
:102F04001BD06D4B1870F32861D900F10C03DBB2B0
:102F1400012B67D9FD2865D06B4B05221A7000235D
:102F2400674A1370674A1370624A1370634A1370D6
:102F3400664A1370664A1370E1E05F4BF0221A7020
:102F44005C4BFF221A7000235C4A13705F4A1370B3
:102F54005F4A137070475C4B05221A70564BF72278
:102F64001A700023564A1370564A1370514A13704C
:102F7400524A1370554A1370554B1B781BB1544B6E
:102F840000221A70BBE00023494A1370504A1370A0
:102F940070474D4B06221A70494B1978464A1170F6
:102FA400F7221A700023474A1370424A1370434AA7
:102FB4001370464A1370464A1370A0E0444B1B78C2
:102FC400002B40F0EF803F4BF7221A70F3E0394BAF
:102FD400FF221A700023394A13703C4A13703C4A8A
:102FE400137070470023334A1370344A1370374AFE
:102FF4001370374A137070472D4A13702F4A137099
:10300400324A1370324A137070472F4B02221A70DF
:10301400284A1070294A10702C4A10702C4A1070DB
:103024006DE00909284B1970224BFF221A70002306
:10303400224A1370254A1370254A13705FE0234A0D
:103044001278002A46D11F4A1070214A12787AB9A0
:10305400F22B11D0F02B1CD009091B4B1970154B06
:10306400FF221A700023154A1370184A137046E0A1
:10307400164BFF221A707047134B03221A70002359
:103084000C4A13700D4A1370104A1370104A1370CF
:1030940035E00D4B04221A70FF230D4A1370054AC4
:1030A40013700023054A1370084A137027E000BF09
:1030B40029670020396F00203A6F00203F710020FB
:1030C4003D7100203B6F0020376D00203E710020D1
:1030D4002D6900203D4A11783D4B19703D4B1978FC
:1030E400117018703C4B04221A70FF233B4A137072
:1030F4003B4A137000233B4A13703B4A13703B4B0B
:103104001B68002B61D03A4B1A68334B1B7802F8CA
:10311400013B384B1968384B914218BF13462C4A6F
:10312400127803F8012B334A1168334A994218BFC5
:103134001A46264B1B7802F8013B2E4B19682E4B7E
:10314400914218BF1346234A127803F8012B294AE7
:103154001168294A994208BF1346254A136000237F
:10316400264A13701F4A13701F4A13701A4B1B7898
:10317400072B01D8042B03D1154B1B78F02B24D932
:10318400174B00221A707047012B3FF4E4AE022B58
:103194003FF4FFAE104B07221A700D4B1B78F02B37
:1031A4003FF40CAF094A1178094B1970094B19788F
:1031B4001170F7221A700023094A1370094A137018
:1031C400094A1370054A137099E770473D7100204E
:1031D4003A6F00203B6F0020376D00202D690020DE
:1031E400396F00203F7100203E7100205C76002082
:1031F40044770020AC0200201C5A002029670020DC
:1032040038B5134B1B68D3B1124B1B68E3B9124B8F
:103214001A68511C196010701A68104B1B689A4286
:103224000ED00F4D0C4CFDF755FC2B6822689342D1
:1032340088BF02F59062D31AB3F57D7FF3D838BD09
:10324400054B084A1A60ECE7FFF72AFEF7E700BFD0
:103254005C7600205876002044770020AC020020E1
:08326400407700201C5A0020F5
:10326C00024B4FF000629A60704700BF00ED00E027
:10327C001D4B9B6803F00C03082B12D00C2B14D0A5
:10328C00042B0AD0184B9B68184AC3F30313184934
:10329C00C95C1368CB4013607047144B154A1A6015
:1032AC00F0E7124B144A1A60ECE70F4BDA68DB6854
:1032BC00C3F30313013302F00302022A0CBF0D49BE
:1032CC000D49B1FBF3F1084AD368D268C3F3062366
:1032DC0001FB03F3C2F3416201325200B3FBF2F380
:1032EC00024A1360CEE700BF00100240B802002073
:0C32FC009CA100080024F40000127A00DD
:10330800024A136843F0200313607047FC760020DC
:10331800064A1368043B1360054A934204D2054ADF
:10332800136843F004031360704700BFB8760020A9
:083338004C740020FC7600201B
:1033400007490B681A1D0A6006498A4202D21A68A8
:103350005A607047044A136843F0040313607047CF
:0C336000B876002030750020FC760020BC
:10336C00044A136853F8041C186843F8040C1368D7
:08337C0019607047B8760020CB
:10338400034A1368191D116053F8042C5A607047DE
:04339400B8760020E7
:10339800074B1A6852F8081C52F8040C42F8080C3B
:1033A8001A68106842F8040C1B681960704700BF5F
:0433B800B8760020C3
:1033BC00074B1A68116852F8040C10601A6852F81E
:1033CC00080C42F8040C1B6843F8081C704700BF3B
:0433DC00B87600209F
:1033E0000D4B1B681A680D49591A6FF00300801ABB
:1033F00010EBA10105D452B1A3EB820212681A604E
:103400007047074A136843F0040313607047043B96
:10341000014A1360704700BFB87600204074002056
:04342000FC76002016
:10342400164B1B681968164A9A1A6FF00300401A63
:1034340010EBA2021AD4043B104A136001291BD9D1
:1034440030B4C1F1010253F82250C1F102029200DA
:103454000A4C23689858134443F8040C0432013985
:10346400F7D1064B1B681D6030BC7047054A1368D2
:1034740043F0040313607047704700BFB876002020
:0834840040740020FC760020DA
:10348C0070B4164B1B681D68154A9A1A6FF003012D
:10349C00491B11EBA2021BD453F8046D0F4A1360A5
:1034AC00012D13D905F1FF3C6FF0030200210B4CE9
:1034BC0023689858134458600131043A6145F7D198
:1034CC00C5F10105054B1B6843F8256070BC7047BE
:1034DC00044A136843F004031360F7E7B87600203E
:0834EC0040740020FC76002072
:1034F400054B1A6852F8041C1068014442F8041C75
:0C3504001A68043A1A607047B87600207C
:10351000024B1A681368013313607047B8760020B5
:10352000054B1A6852F8041C1068091A42F8041C6A
:0C3530001A68043A1A607047B876002050
:10353C00024B1A681368013B13607047B876002081
:10354C00034B1A681368002BBCBF5B4213607047B7
:04355C00B87600201D
:103560000F4B1B681A6882EAE270A0EBE2701F281A
:1035700010DC10B4191F0A4C2160002AA7BF53F8B1
:10358000041C01FA02F253F8042CC24043F8042C44
:1035900010BC7047034A136843F48063136070479C
:0835A000B8760020FC76002043
:1035A800054B1A6852F8041C1068014042F8041CC4
:0C35B8001A68043A1A607047B8760020C8
:1035C400054B1A6852F8041C1068014342F8041CA5
:0C35D4001A68043A1A607047B8760020AC
:1035E000054B1A6852F8041C1068414042F8041C4C
:0C35F0001A68043A1A607047B876002090
:1035FC00024B1A681368DB4313607047B8760020DF
:10360C00024B1A6813685B4213607047B87600204F
:10361C000A4B1B681A6852B153F8041C91FBF2F266
:10362C0043F8042C054A1368043B13607047044AA2
:10363C00136843F400631360704700BFB876002032
:04364C00FC760020E8
:103650000B4B1B681A6862B153F8041C91FBF2F023
:1036600002FB101243F8042C054A1368043B136054
:103670007047044A136843F400631360704700BF47
:08368000B8760020FC76002062
:103688000A4B1B681A685AB153F8041C91FBF2F0F4
:1036980002FB101243F8042C044B1B681860704797
:1036A800034A136843F4006313607047B876002038
:0436B800FC7600207C
:1036BC000B4B1B681A681F2A0CD8012101FA02F265
:1036CC0053F8041C114343F8041C054A1368043BCB
:1036DC0013607047034A136843F4806313607047A8
:0836EC00B8760020FC760020F6
:1036F4000C4B1B681A681F2A0DD8012101FA02F22B
:1037040053F8041C21EA020143F8041C054A136817
:10371400043B13607047044A136843F480631360E6
:0C372400704700BFB8760020FC76002043
:103730000E4B1B681A681F2A11D810B4012101FA18
:1037400002F2194651F8040D084C216030EA0202D9
:1037500014BF0122002243F8042C10BC7047044A15
:10376000136843F480631360704700BFB87600208D
:04377000FC760020C3
:10377400034A1368191D1160024A12685A6070479F
:08378400B8760020BC7600209D
:10378C00074B1A68116852F8040C814214BF0021CF
:10379C00012142F8041C1A68043A1A60704700BFF1
:0437AC00B8760020CB
:1037B000064B1A68116852F8040C091A18BF012147
:1037C00042F8041C1A68043A1A607047B876002060
:1037D000034B1A681368B3FA83F35B0913607047ED
:0437E000B876002097
:1037E400074B1A6852F8041C10688142D4BF0021A8
:1037F400012142F8041C1A68043A1A60704700BF99
:04380400B876002072
:10380800074B1A6852F8041C10688142B4BF0021A3
:10381800012142F8041C1A68043A1A60704700BF74
:04382800B87600204E
:10382C00074B1A6852F8041C10688142ACBF002187
:10383C00012142F8041C1A68043A1A60704700BF50
:04384C00B87600202A
:10385000074B1A6852F8041C106881422CBF0021E3
:10386000012142F8041C1A68043A1A60704700BF2C
:04387000B876002006
:10387400074B1A6852F8041C10688142CCBF00211F
:10388400012142F8041C1A68043A1A60704700BF08
:04389400B8760020E2
:103898000B4B1A6813680B4999420BD801F57C61E8
:1038A8008B4207D852F8042C1A60054A1368083B63
:1038B80013607047044A136843F02003136070478D
:0C38C800B8760020BC320020FC76002006
:1038D400094B1A6813680949994206D801F57C61B5
:1038E4008B4202D81B6813607047054A136843F083
:1038F40020031360704700BFB8760020BC3200205C
:04390400FC7600202D
:10390800104B1A6813686BB1B3F57A7F0ADC13F5AC
:103918007A7F07DB002B0BDD013B0B4951F8233085
:1039280013607047094A136843F480631360704753
:10393800DB4352F8040C044941F82300083A014BD0
:103948001A607047B87600207C420020FC76002080
:10395800044B0A221A60044B1B680BB9034B1A600C
:10396800704700BF8076002000770020D8760020BE
:10397800044B10221A60044B1B680BB9034B1A60E6
:10398800704700BF8076002000770020D87600209E
:1039980006490A6852F804390A602BB104494AF604
:1039A800AA220A60013BFCD1704700BFB87600200C
:0439B800003000409B
:1039BC0005490B6853F80429642000FB02F2034804
:1039CC0002600B60704700BFB87600208476002040
:1039DC00074B4AF6AA221A60064B1A68111D196089
:1039EC00054B1B680549A1FB03135B09536070472A
:1039FC0000300040B8760020847600201F85EB5103
:103A0C0010B4354A136853F80449136033490B68F2
:103A1C0023F001030B60324A936D43F4001393655A
:103A2C00304B586840F4C0705860186820F47030FF
:103A3C001860186840F420301860186A20F0704044
:103A4C001862186A40F080401862586A20F00F0023
:103A5C005862586A40F004005862D86820F47030FC
:103A6C00D860D2F8883023F44053C2F88830630011
:103A7C00DBB24B6014F4807F22D00B464FF0A04297
:103A8C000A610969184A0A431A61144B00229A61A7
:103A9C004FF4E762DA611A6842F001021A60114BC6
:103AAC001B6913F0800F04D00E4B1B6913F4807F3D
:103ABC0004D10E4A136843F04003136010BC7047E6
:103ACC00064A4FF030431361136943F4C22343F0A9
:103ADC0014031361D9E700BFB876002000540040EE
:103AEC0000100240000400480A052400FC76002067
:103AFC00294A136853F804191360284BC8221A601A
:103B0C00274A936913F0050FFBD0254B5A6822F016
:103B1C007F7222F441325A605A6842F0007242F4C9
:103B2C0080325A605A6842F400525A609A6912F014
:103B3C00010F09D19A6912F4756FF7D0194A1368FD
:103B4C0043F0400313607047154BDA6922F4F042DE
:103B5C0022F007021204120CDA61C9B299629A6956
:103B6C0012F0010F09D19A6912F4756FF7D00D4A52
:103B7C00136843F0400313607047094BDA6922F471
:103B8C00F04222F007021204120CDA615A6842F475
:103B9C0080425A60704700BFB876002084770020BE
:083BAC0000540040FC760020EB
:103BB400374B19680868C24301EB82011960354B21
:103BC400994228D300282CD0334BC8221A60334A98
:103BD400936913F0050FFBD0304B5A6822F07F72C3
:103BE40022F441325A605A6842EA004242F00072BA
:103BF4005A605A6842F400525A609A6912F0010FEE
:103C040015D19A6912F4756FF7D0254A136843F0F9
:103C1400400313607047224A136843F0040313609F
:103C240070471F4A136843F480631360704700B5FC
:103C34001A4AD36923F4F04323F007031B041B0C33
:103C4400D3614FF0000C134648F2F87E0CF1010CDE
:103C540051F8042FD2B29A629A6912F0010F0AD174
:103C64009A6912F4756FF7D00D4A136843F0400354
:103C740013605DF804FBDA6902EA0E02DA61844536
:103C8400E4D1064A536843F480435360F1E700BF2C
:103C9400B87600204C740020847700200054004043
:043CA400FC7600208A
:103CA800294BC8221A60294A936913F0050FFBD0E3
:103CB800264B5A6822F07F7222F440325A605A68C2
:103CC80042F0007242F480625A605A6842F48032CC
:103CD8005A605A6842F400525A609A6912F0010F09
:103CE80009D19A6912F0100FF7D0194A136843F0F6
:103CF800400313607047154AD36923F4F04323F057
:103D080007031B041B0CD36113469A6912F0040FB6
:103D180009D19A6912F4756FF7D00D4A136843F008
:103D28004003136070470B4B19680A1D1A60074B54
:103D38005A6AD2B24A60DA6922F4F04222F00702E3
:103D48001204120CDA617047847700200054004096
:083D5800FC760020B876002083
:103D6000344B196851F80409196050B3324BC8221A
:103D70001A60324A936913F0050FFBD02F4B5A6833
:103D800022F07F7222F440325A605A6842F0007288
:103D900042F480625A605A6842EA00425A605A68A5
:103DA00042F400525A609A6912F0010F0FD19A69D9
:103DB00012F0100FF7D0224A136843F0400313604B
:103DC00070471F4A136843F480631360704730B52F
:103DD0001A4AD36923F4F04323F007031B041B0C96
:103DE000D3610024A446134648F2F8754FF0010E43
:103DF0009A6912F0040F0DD19A6912F4756FF7D019
:103E00002CB90F4A136843F04003136030BD094BCF
:103E10001960F6E7DA692A40DA615A6AD2B241F8E3
:103E2000042F0CF1010C74466045E1D1014B19607F
:103E3000ECE700BFB87600208477002000540040F3
:043E4000FC760020EC
:103E4400564B1968564B99422AD30B4653F804092A
:103E5400524A136050B3534BC8221A60524A9369B2
:103E640013F0050FFBD0504B5A6822F07F7222F4F6
:103E740041325A605A6842F480325A605A6842F4B5
:103E840000525A609A6912F0010F15D19A6912F022
:103E9400100FF7D0454A136843F04003136070478E
:103EA400424A136843F00403136070473F4A13689F
:103EB40043F48063136070473B4BDA6922F4F042A9
:103EC40022F007021204120CDA6111F8042C9A622F
:103ED4000839324B1960344B9A6912F0010F09D139
:103EE4009A6912F0100FF7D0304A136843F0400378
:103EF400136070472C4BDA6922F4F04222F0070277
:103F04001204120CDA615A6822F07F7222F44032F1
:103F14005A605A6842F0007242F480625A605A68E9
:103F240042EA00425A605A6842F400525A609A695E
:103F340012F0010F09D19A6912F0100FF7D01B4A41
:103F4400136843F040031360704730B50024A4465F
:103F5400154B48F2F8754FF0010E9A6912F0040FF0
:103F64000DD19A6912F4756FF7D02CB90F4A136802
:103F740043F04003136030BD084B1960F6E75A6AFA
:103F8400D2B241F8042FDA692A40DA610CF1010C4B
:103F940074466045E1D1014B1960ECE7B876002026
:103FA4004C7400208477002000540040FC760020EC
:103FB4000A4B1A68136803F140400949884207D83C
:103FC40052F8042C1A60054A1368083B13607047C2
:103FD400044A136843F4806313607047B876002082
:083FE400000C0610FC76002021
:103FEC00084B1B681A6802F140400749884202D806
:103FFC0012681A607047054A136843F480631360B3
:10400C00704700BFB8760020000C0610FC7600202C
:10401C00114B1A68136803F14040104988420ED8BE
:10402C0052F8042C1F2A10D8012101FA02F2196847
:10403C0011431960084A1368083B13607047084A1B
:10404C00136843F4806313607047054A136843F4A4
:10405C0080631360704700BFB8760020000C061018
:04406C00FC760020BE
:10407000114B1A68136803F14040104988420FD869
:1040800052F8042C1F2A11D8012101FA02F21968F2
:1040900021EA02011960084A1368083B136070475F
:1040A000074A136843F4806313607047044A136837
:1040B00043F4806313607047B8760020000C06104C
:0440C000FC7600206A
:1040C400134B1B681A6802F140401249884213D806
:1040D40053F8041C1F2915D810B4012000FA01F16B
:1040E40010681A1F0A4C2260014214BF01220022E8
:1040F40043F8042C10BC7047074A136843F48063E8
:1041040013607047044A136843F480631360704774
:0C411400B8760020000C0610FC7600209D
:1041200010B408490A6852F804490748074B1B684D
:1041300003F18043013B00EB830340F824300A6025
:1041400010BC7047B8760020BC0200200C7700201D
:10415000044A1368191D1160034A126852F8042CAE
:0C4160005A607047B8760020C07600203E
:10416C00084B4AF6AA221A60074B1B681A68131FE1
:10417C0052F8042C8D2A0CBF043B5B68034A136075
:10418C00704700BF00300040C0760020EC76002065
:10419C00024B1B681A68024B1A607047C0760020ED
:0441AC00EC7600208D
:1041B000064B1B681A6822B9054A12681168054A3D
:1041C0001160043B014A1360704700BFB8760020BD
:0841D000C0760020EC7600200F
:1041D800164B1B681968164A1160164A934218D97B
:1041E800154A1268022A07D0043B104A1360134A82
:1041F8001368013B13607047104A1168104A12682F
:104208009142F1D10E4A002111600B4A032111603D
:10421800EAE7074B00221A60074B1B68022B00D005
:104228007047054B03221A60FAE700BFC0760020EA
:10423800EC76002040730020A8020020E0760020E1
:0442480018770020C3
:10424C00054B00221A605A609A6003F10C00034976
:10425C000860DA60704700BF40740020B876002018
:0C426C00014B03221A607047A8020020DA
:0C427800014B01221A607047A8020020D0
:0C428400014B00221A607047A8020020C5
:1042900010B50023404A1360404A1360404A13603F
:1042A000404A1360404A1360404A01211160404A6D
:1042B0001360404A1168404A1160404A117819B1B0
:1042C00001331832A82BF9D13D4A13603D4AD2F888
:1042D000FC2F7D2A4DD03C4940F6FF321446013A6E
:1042E00051F8040D7D2834D0002AF7D10022374937
:1042F0000A6037490A60314A03EB430302EBC30308
:1043000002F57C62934228BF00240AD200240021D7
:10431000304A43F8041B9342FBD340F6FE339C42E1
:104320000AD82D4B03EB8403002140F6FE3243F8FC
:10433000041F01349442FAD9284A294B1A600023F9
:104340001360284A28491160284A1360FFF77EFF4E
:1043500010BD002ACAD01D4A14601D4A1460174AB5
:1043600003EB430302EBC30302F57C629342CED31B
:10437000D3E74FF4406215490A6015490A600F4AB5
:1043800003EB430302EBC30302F57C62934238BFA5
:104390004FF44064BBD3CFE70477002000770020C0
:1043A000F876002014770020E0760020A802002094
:1043B0007C760020D876002080760020BC32002059
:1043C000DC760020BC220020B83200200C770020D0
:1043D000087700207C420020B802002040730020B3
:1043E000C0760020EC760020BC020020FC76002085
:1043F000054A1368191D116004490A68101D0860F8
:1044000052685A60704700BFB8760020EC760020F2
:10441000054A1368191D116004490A68101D0860D7
:10442000526812685A607047B8760020EC76002017
:10443000064B1A68111D1960054B19680968526806
:1044400011601A68043A1A60704700BFEC760020C9
:04445000B87600201A
:10445400084B1B681A6842B1074A126804320649BD
:104464000A60043B034A13607047034A12685268A7
:0C447400F5E700BFB8760020EC760020D1
:10448000084B1B68196853F8042C9142064A1268BD
:104490000CBF0432526804490A60043B014A1360AD
:0C44A000704700BFB8760020EC760020CA
:1044AC00084B1B68196853F8042C9142064A126891
:1044BC00CCBF0432526804490A60043B014A1360C1
:0C44CC00704700BFB8760020EC7600209E
:1044D800084B1B68196853F8042C9142064A126865
:1044E800B4BF0432526804490A60043B014A1360AD
:0C44F800704700BFB8760020EC76002072
:10450400024B1A6852681A60704700BFEC760020AC
:10451400054A1368191D116004490A68101D0860D2
:1045240052685A60704700BFC0760020EC760020C5
:104534000C4B1B681B6863B10B4A1368043B136084
:104544000A4A136808331360064A1368043B13606D
:104554007047074B4AF6AA221A60044B1A6852683D
:104564001A60F1E7B8760020C0760020EC760020CF
:0445740000300040D3
:104578000C4B1B681B6863B90B4A1368043B136038
:104588000A4A136808331360064A1368043B136029
:104598007047074B4AF6AA221A60044B1A685268F9
:1045A8001A60F1E7B8760020C0760020EC7600208B
:0445B800003000408F
:1045BC00044B4AF6AA221A60034B1A6852681A6016
:0C45CC00704700BF00300040EC7600207B
:1045D8000B4B1A6802F1100119600A490B6853F86D
:1045E800080CD06053F8040C906053F80C09506024
:1045F8000B6005490B68181D08605B6813617047FC
:0C460800C0760020B8760020EC76002080
:104614001C4B1B6853F8042C53F8080C53F80C1C5F
:104624000A44002916DB90420CDD174B4AF6AA21F6
:104634001960144B1B6843F8042C144B1A68526815
:104644001A607047103B0F4A1360104A136808330E
:104654001360704790420CDA0B4B4AF6AA2119609A
:10466400084B1B6843F8042C084B1A6852681A60FC
:104674007047103B034A1360044A136808331360FD
:10468400704700BFC076002000300040EC76002068
:10469400024A1368043B1360704700BFC0760020D1
:1046A400024A1368103B1360704700BFC0760020B5
:1046B40007490A6852F804390A60013BB3F5007FE0
:1046C40023BF044A136843F48063034A13607047AA
:0C46D400B8760020FC7600203077002033
:1046E000064B1B68064AD25CFF2A06D001320449F9
:1046F000CA540449CA5C0132CA547047307700205A
:084700003C6F0020346B002027
:10470800064B1B68064AD25C32B1013A0449CA54C6
:104718000449CA5C013ACA54704700BF3077002088
:084728003C6F0020346B0020FF
:10473000054B064903F50070002203F8012F01F82C
:10474000012F8342F9D170473B6F0020336B00206B
:10475000094A136853F804191360A1F11803B3F55B
:10476000F47F02D8054B19607047054A136843F47B
:1047700080631360704700BFB87600202C7700205C
:04478000FC760020A3
:1047840010B5044C23681878FBF77CFF2368043BBE
:08479400236010BDB87600207F
:10479C0008B5104B1B6803B108BD2020FBF76EFF5A
:1047AC002D20FBF76BFF3E20FBF768FF4420FBF747
:1047BC0065FF4220FBF762FF4720FBF75FFF2020DD
:1047CC00FBF75CFF034B01221A60034B00221A60BB
:0C47DC00E2E700BFA80200207876002071
:1047E80008B5104B1B6883B10F4B1B686BB10F4B9F
:1047F8001B68ABB10E4A1368191D11600D4A127877
:104808005A600A4B00221A600AE0FDF725FA0346AF
:104818000028FAD006490A68101D0860DBB2536008
:1048280008BD00BFA8020020F87600207C76002092
:08483800B8760020BE770020D5
:1048400010B5064C2368186806F08DFD2020FBF794
:104850001BFF2368043B236010BD00BFB876002017
:1048600008B50E4B1B68102B07D00D4B1B68186842
:1048700000F160420B4B9A420CD8094B1B68186838
:1048800006F071FD2020FBF7FFFE054A1368043B8C
:10489000136008BDFCF7BAFFF4E700BF8076002084
:0848A000B8760020FF0B063082
:1048A8002DE9F04186B0294B93E8070006AB03E9F0
:1048B8000700274B93E803000190ADF808105B2030
:1048C800FBF7DEFE234B1B68234A93420CD0224A97
:1048D80093420DD319D9151D0424A2F10C06DFF853
:1048E8007C8006F10C0722E001A806F0D0FC0CE061
:1048F80003A806F0CCFC1A4B00221A605A609A6092
:1049080003F10C0013490860DA605D20FBF7B8FE7C
:1049180006B0BDE8F081286806F021FD2020FBF7ED
:10492800AFFE01340B4B1B680435BB42EDD99B1B12
:10493800B4EBA30FE9D82020FBF7A2FED8F800308B
:10494800102BE8D02868FCF75DFFE7E718AD0008F2
:1049580024AD0008B87600204C7400208076002032
:044968004074002077
:10496C002DE9F04784B0384A01AB07CA03C31A706B
:10497C002020FBF783FE354B1B68002B5CD0344D9D
:10498C0000273E464FF02008DFF8C8A0DFF8BC90A7
:10499C0017E04046FBF772FE15E0D5F8053013F032
:1049AC00404F21D14046FBF769FE4046FBF766FEBF
:1049BC0001360137052F36D81835D9F80030B342F7
:1049CC0039D9092EE5D93046FCF71AFF3A20FBF706
:1049DC0055FEA5F1100414F8010F0028DDD0FBF7EB
:1049EC004DFEAC42F7D1D8E701A806F04EFCDAF840
:1049FC000030102B12D0D5F80100FCF701FF404617
:104A0C00FBF73CFE4020FBF739FE681C80B206F039
:104A1C00A4FC2920FBF732FE0237C3E7D5F80100CE
:104A2C0006F09BFCEBE70D20FBF728FE4046FBF75E
:104A3C0025FE0027C0E717B904B0BDE8F0870D20AC
:104A4C00FBF71CFEF8E700BFF4B00008DC76002092
:084A5C00CB320020807600201F
:104A64002DE9F04184B0264B6C460FCB07C423706C
:104A7400244A136853F804591360B5F5007F07D925
:104A8400214A136843F48063136004B0BDE8F081E5
:104A9400684606F0FEFB1D4C20680130FCF7B4FEAE
:104AA4003A20FBF7EFFD2020FBF7ECFD5620FBF747
:104AB400E9FD3D20FBF7E6FDD4F80080144B13F824
:104AC4000800FCF7A1FE08F10104B4F5007F13D03F
:104AD400012D11D00E4B1C4403F2FF172C26434426
:104AE4001D443046FBF7CEFD2078FCF78DFEBC421A
:104AF40002D00134AC42F4D10D20FBF7C3FDC4E76E
:104B040000B10008B8760020FC7600203077002041
:044B14003C6F0020D2
:104B180010B5044C2368186806F0CDF82368043BE8
:084B2800236010BDB8760020E7
:104B300010B5044C23681878FBF700FF2368043B8A
:084B4000236010BDB8760020CF
:104B4800F8B50C4A136853F8047913605FB1C7F1DC
:104B58000104A4003D4616463368185DFBF7EAFEDB
:104B68000434013DF8D1034A1368A3EB87031360AB
:084B7800F8BD00BFB876002073
:104B800008B5154B1B681B68B3F5805F0CD2134B3F
:104B90001B6813F0010F0DD00F4A136853F8040976
:104BA0000E498860136008BD0D4A136843F48063A2
:104BB0001360F8E70B4AD36C43F48033D364074B9C
:104BC0001A6802F001121A601A6842F001021A60B3
:104BD000FBF76CFCE0E700BFB8760020000800504F
:084BE000FC76002000100240E9
:104BE80008B5154B1B681B68B3F5805F0CD2134BD7
:104BF8001B6813F4803F0DD00F4A136853F804095B
:104C08000E494861136008BD0D4A136843F4806378
:104C18001360F8E70B4AD36C43F48033D364074B33
:104C28001A6802F001121A601A6842F480321A6097
:104C3800FBF738FCE0E700BFB8760020000800501A
:084C4800FC7600200010024080
:104C50002DE9F04F85B02F4A02AB92E8030083E8BC
:104C600003002D4A92E8030000908DF804101846C6
:104C700006F011FB0D20FBF707FDDFF8A0900127E0
:104C80004FF002084FF0000A20264FF0230B2CE0D3
:104C9000FBF7FAFC013415F8010B0028F8D1062CBB
:104CA00005D83046FBF7F0FC0134072CF9D1584603
:104CB000FBF7EAFC384606F0FAFA3046FBF7E4FC6C
:104CC0003046FBF7E1FC3046FBF7DEFC972F12D0B5
:104CD0000AF1010ABAF1050F13D008F101080137F2
:104CE00009F10809B8F1AB0F11D03046FBF7CCFC45
:104CF0004D460024CFE70D20FBF7C6FC684606F0C2
:104D0000CAFA0D20FBF7C0FC4FF0000AE5E705B03A
:104D1000BDE8F08F10B1000818B10008CCA500085C
:104D20002DE9F0478CB001AC334D0FCD0FC40FCD42
:104D30000FC495E8070003C424F8022B120C22705C
:104D40002E4B1B6863B12E4B1B684BB12C4B0022C2
:104D50001A602C4A1368191D11602B4A12685A6098
:104D6000284A136853F80459136045F00055274B3F
:104D70009D4207D9264A136843F4806313600CB040
:104D8000BDE8F0870D20FBF77FFC01A806F083FA51
:104D9000284605F066FF05F1800803264FF00D0A4E
:104DA0004FF03A097C2714E02468200E06F07FFAC1
:104DB000C4F3074006F07BFAC4F3072006F077FA45
:104DC000E0B206F074FA3846FBF75EFC0435454560
:104DD0000ED02C460136042EE6D15046FBF754FC8B
:104DE000284605F03EFF4846FBF74EFC0026DBE771
:104DF0000D20FBF749FCC2E720B10008F87600203F
:104E000014770020B876002010770020807F0020E3
:044E1000FC7600200C
:104E140070B5D2B0974B93E803005090ADF84411AD
:104E2400090C8DF84611944B4DAE93E8070086E8C3
:104E34000700924B93E803004B90ADF83011090C36
:104E44008DF832118E4A49AB92E8030083E80300DF
:104E540044AC8C4D0FCD0FC42B6824F8023B1B0CC3
:104E64002370894A41AB07CA03C31A803CAC874DFF
:104E74000FCD0FC42B6824F8023B1B0C2370844B0A
:104E840038AC0FCB07C42370824A35AB07CA03C3BF
:104E94001A80814A32AB07CA03C31A807F4A30ABF7
:104EA40092E8030083E803007D4A2EAB92E80300F6
:104EB40083E803007B4A2BAB07CA03C31A707A4BFF
:104EC40093E803002990ADF8A810090C8DF8AA10F6
:104ED400764A26AB07CA03C323F8022B120C1A70B6
:104EE400734A23AB07CA03C31A70724B93E80300D7
:104EF4002190ADF88810090C8DF88A106E4B209320
:104F04006E4B93E803001E90ADF87C106C4A1BAB0B
:104F140007CA03C31A706B4A18AB07CA03C31A70D3
:104F2400694B93E803001690ADF85C10674B93E867
:104F340003001490ADF85410654B93E803001290ED
:104F4400ADF84C10090C8DF84E10624A0FAB07CA2D
:104F540003C323F8022B120C1A700AAC5E4D0FCD5A
:104F64000FC42B6823605D4A07AB07CA03C323F849
:104F7400022B120C1A705A4A04AB07CA03C31A70E4
:104F840001AB584A07CA83E807004420FBF77AFBC1
:104F94006120FBF777FB7420FBF774FB6120FBF7C0
:104FA40071FB50A806F075F94F4805F058FE5220E1
:104FB400FBF768FB6520FBF765FB7420FBF762FBDE
:104FC4007520FBF75FFB7220FBF75CFB6E20FBF7A1
:104FD40059FB50A806F05DF9444805F040FE304600
:104FE40006F057F9424805F03AFE5520FBF74AFB14
:104FF4007320FBF747FB6520FBF744FB7220FBF7AC
:1050040041FB3D20FBF73EFB3A4805F028FE0D200E
:10501400FBF738FB384B1B68F3B149A806F039F9A4
:10502400354B1B68E3B944A806F033F9334B1B68CE
:10503400002B65D000242F4E304D2B68013B03EB31
:10504400430306EBC303185D002865D0FBF71AFB86
:105054000134102CF1D15FE04BA806F01AF9DCE71B
:105064002320FBF70FFB244B18683030C0B2FBF74A
:1050740009FBD8E7ACA10008B4A10008C0A100084E
:10508400C8A10008D0A10008E4A10008F0A100080C
:1050940004A2000814A2000820A200082CA2000800
:1050A40034A200083CA2000848A2000850A200084C
:1050B4005CA2000868A200084F46460070A20008DF
:1050C40078A2000884A2000890A2000898A2000810
:1050D400A0A20008A8A20008B4A20008C8A2000860
:1050E400D4A20008E0A200084C7400204073002001
:1050F400BC020020BC320020907700201C770020E6
:105104006E20FBF7BFFA6F20FBF7BCFA6E20FBF7AB
:10511400B9FA6520FBF7B6FA3CA806F0BAF8BC4B1E
:1051240018683030C0B2FBF7ADFA0D20FBF7AAFACD
:1051340041A806F0AEF8B74B1868B74BA3FB003094
:10514400800CFCF761FB4D20FBF79CFA4820FBF731
:1051540099FA7A20FBF796FA38A806F09AF8AF4C39
:105164002068FCF751FB23681F2B00F085810B2B73
:1051740000F08C81A94B1B68132B00F08E81A74B88
:105184001B68262B00F08D81A44B1B68392B00F083
:105194008C813020FBF776FA3020FBF773FAA04BB2
:1051A4001B6843B99A4B1B6823F00203012B02D0FE
:1051B40032A806F06EF835A806F06BF8994B18681B
:1051C400002840F076816120FBF75CFA6C20FBF745
:1051D40059FA6C20FBF756FA30A806F05AF8924BAD
:1051E4001868FCF711FB2C20FBF74CFA8F4B1B685B
:1051F400102B00F061818E4B1868FCF705FB2C2006
:10520400FBF740FA8B4B1868FCF7FEFA0D20FBF70E
:1052140039FA2EA806F03DF8874B1C68002C40F0A4
:1052240057810020FCF7F0FA2BA806F032F8834BE4
:1052340018680028C0F278817C4B1B68102B00F0A2
:105244007781FCF7E1FA29A806F023F87C4B18686B
:105254000028C0F27081754B1B68102B00F06F8121
:10526400FCF7D2FA26A806F014F8764B1C68002C3A
:1052740040F068810020FCF7C7FA23A806F009F87B
:10528400714B18680028C0F28981684B1B68102B89
:1052940000F08881FCF7B8FA21A805F0FAFF6B4BFF
:1052A40018680028C0F28181604B1B68102B00F045
:1052B4008081FCF7A9FA0D20FBF7E4F91EA805F09C
:1052C400E8FF634B1B6FB3F1FF3F40F079814FF070
:1052D40090435B6913F0020F40F06E8112A805F051
:1052E400D8FF3120FBF7CEF91BA805F0D2FF584BAD
:1052F400D3F88830B3F1FF3F40F075814FF090430D
:105304005B6913F0100F40F06A8112A805F0C1FF29
:105314003220FBF7B7F918A805F0BBFF4C4BD3F8C4
:10532400A030B3F1FF3F40F072814A4B5B6913F048
:10533400800F40F0688112A805F0ABFF3320FBF723
:10534400A1F90D20FBF79EF90FA805F0A2FF0D208F
:10535400FBF798F90AA805F09CFF3F4C2068013040
:1053640005F0ABFC5420FBF78DF97820FBF78AF9A4
:105374003D20FBF787F92368384AD05C05F09DFC93
:105384004620FBF77FF96920FBF77CF96E20FBF7D9
:1053940079F96120FBF776F96C20FBF773F93D206E
:1053A400FBF770F923682E4AD05C05F086FC07A849
:1053B40005F06FFF2B4D2C682B4BA3FB04346409C1
:1053C4002046FCF721FA2E20FBF75CF92868274BCE
:1053D400A3FB003004EB84046400C4EBD000FCF7AE
:1053E40013FA04A805F055FF214B1868FCF70CFAD2
:1053F40001A805F04EFF1F4B1868FCF705FA292099
:10540400FBF740F90D20FBF73DF952B070BD00BF2A
:1054140088770020B802002083DE1B4380770020B9
:10542400AC770020A8770020A076002080760020AA
:10543400A8760020A4760020F4760020D4760020FC
:10544400D0760020F0760020CC760020C8760020AC
:10545400BC32002000040048307700203C6F00205C
:10546400346B0020247700201F85EB51CDCCCCCCAD
:105474002C770020347700203220FBF703F9352005
:10548400FBF700F93020FBF7FDF888E63520FBF741
:10549400F9F83220FBF7F6F86CE63220FBF7F2F865
:1054A4006DE63420FBF7EEF86EE63620FBF7EAF8FB
:1054B4006FE6FCF7A9F98FE65D4B186805F051FF1C
:1054C4002C20FBF7DFF85B4B186805F04AFF9DE6DC
:1054D4004FF4FA6303FB04F5574EB6FBF5F630467A
:1054E400FCF792F906FB04F0544B554C03FB0044C3
:1054F4002E20FBF7C7F8B4FBF5F63046FCF784F929
:1055040005FB164303EB83035B00B3FBF5F005FBDC
:10551400103303EB83035B00B3FBF5F3042B88BF69
:105524000130FCF771F97FE620A805F0B2FE8AE6A7
:1055340005F017FF87E620A805F0ABFE92E605F01C
:1055440010FF8FE64FF4FA6303FB04F53A4EB6FB03
:10555400F5F63046FCF758F906FB04F0374B384CA7
:1055640003FB00442E20FBF78DF8B4FBF5F6304620
:10557400FCF74AF905FB164303EB83035B00B3FB1B
:10558400F5F005FB103303EB83035B00B3FBF5F38A
:10559400042B88BF0130FCF737F96EE620A805F02C
:1055A40078FE79E605F0DDFE76E620A805F071FECA
:1055B40081E605F0D6FE7EE62D20FBF763F88DE646
:1055C40016A805F066FE1F4B1868FCF71DF914A811
:1055D40005F05FFE1C4B186FFCF716F984E62D20CE
:1055E400FBF750F891E616A805F053FE174B186820
:1055F400FCF70AF914A805F04CFE134BD3F8880005
:10560400FCF702F987E62D20FBF73CF893E616A891
:1056140005F03FFE0E4B1868FCF7F6F814A805F0E9
:1056240038FE094BD3F8A000FCF7EEF889E600BF7A
:10563400A8760020A4760020006CDC02E0B1FFFF15
:1056440000389C1C90760020BC3200208C76002010
:045654008876002034
:1056580010B59CB00DF1500C2F4C0FCCACE80F00DE
:1056680094E80F00ACE80700ACF800304A222B4958
:1056780001A805F07EFC2A4A136853F80449136010
:10568800112C1BD0192C31D0312C03D11F240B2CF9
:1056980019D003E0382C08BF262410D1132C12D0BF
:1056A8001F2C10D0262C0ED0392C0CD0602C0AD0F0
:1056B8001C4A136843F4806313602AE00B24572CB8
:1056C80008BF392413D1184B1B6823F00203012BA0
:1056D80012D001A805F0DBFD144B1C60144B1C60B4
:1056E800FBF7CCFA134B00221A600FE01324962C18
:1056F80008BF6024E7D0CAE714A805F0C8FD0D204C
:10570800FAF7BEFF0A4B1C60FAF742FF0D20FAF7C2
:10571800B7FF1CB010BD00BF38AD000858AD000879
:10572800B8760020FC76002088770020B07700202B
:0857380080770020AC7700200F
:1057400010B58EB0EC46154C0FCCACE80F000FCC6A
:10575000ACE80F000FCCACE80F0094E803004CF865
:10576000040BACF800100E4B1B681B68102B0ED8F6
:105770000C4A13603BB10A4A1368043B1360FBF701
:1057800081FA0EB010BD684605F085FDF3E7064AC4
:10579000136843F480631360F3E700BFB0AD000803
:0C57A000B8760020A8770020FC760020DE
:1057AC0008B50A490A6852F804390A607F2B05D9F2
:1057BC00074A136843F48063136008BD03EB83034B
:1057CC005B00044A1360FBF757FAF6E7B876002043
:0857DC00FC7600202477002078
:1057E40008B5094A136853F804191360602905D9E8
:1057F400064A136843F48063136008BD044B1960C0
:10580400FBF73EFAF9E700BFB8760020FC760020EB
:0458140034770020C5
:1058180008B5084A136853F804091360FF2805D926
:10582800054A136843F48063136008BDC0B204F0EE
:0C583800DDFAFAE7B8760020FC760020CC
:1058440070B5184C2668184A136853F80459136045
:10585400C5F3074004F0CCFA236801332360B3F5A1
:10586400007F06D9114A136843F4806313602660ED
:1058740070BDC5F3072004F0BBFA0A4A136801336C
:105884001360B3F5007F07D9084A136843F48063B3
:105894001360044B1E60EBE7E8B204F0A9FA014B75
:1058A4001E60E5E730770020B8760020FC76002003
:1058B40038B5204A136853F8045913601E4B1A680C
:1058C400D41C1C60B4F5007F07D91C490B6843F451
:1058D40080630B60184B1A6038BDC5F3074004F0B1
:1058E40087FA154A136801331360B3F5007F07D9AB
:1058F400124A136843F4806313600F4B1C60EBE798
:10590400C5F3072004F074FA0B4A136801331360DB
:10591400B3F5007F07D9094A136843F48063136021
:10592400054B1C60D8E7E8B204F062FA024B1C6035
:10593400D2E700BFB876002030770020FC76002044
:1059440010B5094A136853F804491360FF2C05D9AC
:10595400064A136843F48063136010BDFEF7A8FE83
:10596400E0B204F045FAF8E7B8760020FC760020AF
:1059740008B50C4A136853F804091360FF2804D8C7
:10598400094B1B68B3F5FF7F05D9084A136843F434
:105994008063136008BD0133034A1360C0B204F08E
:1059A40027FAF7E7B876002030770020FC7600204D
:1059B4002DE9F843154A136853F804691360EEB1EE
:1059C400134BD3F80090C9F50073B34216D3114BAF
:1059D40013F8098000250E4C40F2FF1723680133A9
:1059E4002360404604F004FA2368BB4202D0013528
:1059F400AE42F3D1064BC3F8009004E0064A1368A4
:105A040043F480631360BDE8F88300BFB8760020D8
:0C5A140030770020346B0020FC7600206E
:105A20001A490A6852F80439013B0A605F2B27D8EB
:105A300010B5980803F00303590200F5803E0EF1FB
:105A4000280E4FEACE2E124A531E02F2FF74C2F104
:105A5000010C0EEB030212F80C20D24303F8012FC5
:105A6000A342F6D10B4B0C4A0A4403F5007413F819
:105A7000011F02F8011FA342F9D1FBF74BFE10BD35
:105A8000064A136843F4806313607047B8760020B9
:105A90001C5200203B6F00201B520020FC7600208F
:105AA00024490A6852F804390A60602B12D82DE99B
:105AB000F041ABB9204B03F50071002203F8012F30
:105AC0008B42FBD1DFF874801B4D08F5007644460D
:105AD0001B4F22E01B4A136843F480631360704736
:105AE000013B9A0802F58032283203F00303590281
:105AF00001EBC221144BC91A03F500705A58D24366
:105B000043F8042B8342F9D1DCE7601EA0EB0800C8
:105B100080B204F03FF9B4420AD0013415F8013FD5
:105B200022789A42F7D03A68002AEED12370F2E741
:105B3000BDE8F081B8760020336B00203B6F002079
:0C5B400024770020FC760020346B00204D
:105B4C002DE9F84F3F4A13681E6853F8045C53F86C
:105B5C00081C0C3B1360DEB13B4B1C68C4F5007396
:105B6C00B34215D36B1EB3F5007F11D260290FD849
:105B7C0071BBA3199C4210D2651E344F2F44344B79
:105B8C001D444FF00008DFF8CCA0DFF8BC9012E009
:105B9C00314A136843F480631360BDE8F88FA0B2F8
:105BAC0004F0F2F8B4F5007FF7D00134D9F80030E6
:105BBC003344A342F1D907F8018F01352B78002B20
:105BCC00F3D0DAF80030002BE9D185F80080E9E752
:105BDC0001398D0805F58032283201F003014D02A0
:105BEC0005EBC22505F5007B1D44A3199C42D4D2BC
:105BFC00671E164B07EB0308154B1F44DFF854A028
:105C0C00DFF844900BE03B70B4F5007FC5D0AB459A
:105C1C00C3D00134D9F800303344A342BDD915F8B0
:105C2C00013BDB43DBB208F8013F01373A789A427B
:105C3C00EFD0DAF80020002AE5D0A0B204F0A4F8E6
:105C4C00E2E700BFB876002030770020346B0020EC
:0C5C5C003C6F002024770020FC76002024
:105C680070B5BAB0A54B93E803003890ADF8E410CE
:105C7800090C8DF8E610A24B93E803003690ADF8B6
:105C8800DC10090C8DF8DE109E4A33AB07CA03C33B
:105C980023F8022B120C1A709B4A30AB07CA83E810
:105CA80007009A4A2DAB07CA03C323F8022B120C2C
:105CB8001A70974B29AC0FCB07C423800DF1900CB9
:105CC800944C0FCCACE80F0023682CF8023B1B0C5B
:105CD8008CF800300DF1780C8F4C0FCCACE80F002D
:105CE80094E803004CF8040B8CF800108B4B1AACAA
:105CF8000FCB84E80F0015AC894D0FCD0FC42B686E
:105D0800236010AC874D0FCD0FC42B6823800DF195
:105D1800280C854C0FCCACE80F0094E803004CF835
:105D2800040B8CF8001005AC804D0FCD0FC42B6808
:105D380023806C467E4D0FCD0FC42B6823807D4B8E
:105D48001B687D4A9342C0F093807C490A6842F000
:105D580004020A607A4A934204D2784A136843F0EC
:105D680004031360774B1B68B3B1774B186800EBDB
:105D78004002D100754A4B1E13440F320A440021D9
:105D880003F8011F9342FBD1704B00EB400203EB79
:105D9800C2020021116151616A4B00221A606C4BEA
:105DA8001B687BB114462026694D3046FAF768FC1B
:105DB80001342B68A342F8D85E20FAF761FC0D2065
:105DC800FAF75EFC38A805F062FA5C4C206805F02A
:105DD80084FA3D20FAF754FC236813F0010F69D1C7
:105DE800564B1B6813F0020F68D1544B1B6813F015
:105DF800040F67D1514B1B6813F0080F66D14F4B46
:105E08001B6813F0400F65D14C4B1B6813F0200F33
:105E180064D14A4B1B6813F0800F63D1474B1B6852
:105E280013F4807F62D1454B1B6813F4007F61D166
:105E3800424B1B6813F4806F40F092803F4B1B6805
:105E480013F4006F40F0908036A805F020FA404B1C
:105E5800186804F038FF2920FAF712FCFEF714FA44
:105E68000D20FAF70DFC3B4B00221A603AB070BDCA
:105E7800334A9342FFF471AF304B1B68002B7FF419
:105E880071AF304B1B68002B72D1334B1B68012B51
:105E9800E6D02020FAF7F4FB6F20FAF7F1FB6B202D
:105EA800FAF7EEFB2D4B1B68102BD9D14820FAF7D7
:105EB800E7FBD5E733A805F0EAF991E730A805F044
:105EC800E6F992E72DA805F0E2F993E729A805F08D
:105ED800DEF994E724A805F0DAF995E71EA805F09D
:105EE800D6F996E71AA805F0D2F997E710A805F0B1
:105EF800CEF998E715A805F0CAF999E7F4AD0008B6
:105F0800FCAD000804AE000810AE00081CAE000886
:105F180028AE000838AE00084CAE000864AE000891
:105F280074AE000888AE00089CAE0008B4AE000845
:105F3800C8AE0008B876002030750020FC76002036
:105F48004C74002000770020DC760020BC32002052
:105F580068760020147700200477002080760020DF
:105F68000AA805F094F969E705A805F090F96BE728
:085F7800684605F08CF973E79F
:105F800038B5FBF76DFE0446002800F0D180C0B2A2
:105F90006B4B1B683BB16B4B1B6823B16A4B187092
:105FA0006A4B01221A600A2800F0BF80022840F2E2
:105FB000BE80644B1C684CB9092808BF2020644B84
:105FC0001B683F2B02D9202800F09A80282815D082
:105FD0002F283CD01B2863D1002C00F0A9800D2075
:105FE000FAF752FB5A4B1A685A4B20219954134422
:105FF00000215970584B1A60022499E0574B1C68D5
:106000000CB1002494E0FAF73FFBFBF729FE0028CF
:10601000FBD0C0B220280BD04D490B684D4A282533
:10602000D5541A44507002330B60FAF72DFB7FE011
:10603000474B1B680133494A13600820FAF724FBD9
:106040002020FAF721FB0820FAF71EFB70E0434BF3
:106050001C680CB100246BE0FAF716FBFBF700FE9E
:106060000028FBD0C0B22F280BD039490B68394A21
:106070002F25D5541A44507002330B60FAF704FBF5
:1060800056E0334B1B680133344A13600820FAF79B
:10609000FBFA2020FAF7F8FA0820FAF7F5FA47E0B9
:1060A000092847D0122847D0082818D12B4B1D6843
:1060B0000DB100243CE0264B1C68002C38D0631E38
:1060C000234A13602024234AD454FAF7DDFA2046E9
:1060D000FAF7DAFA0820FAF7D7FA2C4628E00D2862
:1060E00016D11B4B1B685BB9194B1A68194B202141
:1060F0009954134400215970174B1A60012417E07A
:10610000164B1B68012BEFD00D20FAF7BDFAEBE719
:10611000124B1C6894B90E4D2B680E4AD054FAF7F6
:10612000B3FA2B6801332B6002E0002400E0002466
:10613000204638BD0324FBE70424F9E70024F7E7F1
:10614000A8020020F8760020BE7700207C76002090
:1061500070760020407500207476002004770020BF
:10616000164B1868164B1A5C202A0AD103441449AE
:10617000C1F10101C81813F8012F202AFAD00F4BE2
:106180001860AAB110B40F4901440F4C002311F854
:10619000012F202A04D004F8012B0133102BF6D153
:1061A000094A0021D1540344084A136010BC7047C7
:1061B000054B00221A70054B186070476876002066
:1061C000407500203F750020E475002070760020A7
:1061D0002DE9F04F87B00F4601380DF10809494607
:1061E000002505E011F8013CFBB10135102D0CD064
:1061F00010F8013F01F8013BA3F16102D2B2192A64
:10620000F0D8203B01F8013CEFE700238DF8173070
:106210009DF808302D2B0FD1264B00221A60012D3E
:1062200042D9012301931E460EE000238DF817305A
:106230009DF808302D2B29D01E4B00221A6001201A
:106240007DB3002301931E461A4BD3F8008006ABA2
:106250001E44113E4FF0000A4FF0010B3446394600
:1062600016F8010F05F08BF8B0F1FF3F12D007FBD5
:106270000808DA460234A4EB0904AC42EED30D4B15
:10628000C3F80080019B7BB901200AE0012DC3D136
:10629000002006E0BAF1000F02D0064BC3F80080E0
:1062A000002007B0BDE8F08F024A13685B4213601C
:0862B0000120F6E76C760020E6
:1062B80008B5364B187800285CD01A4600230133FD
:1062C80012F8011F0029FAD12D2811D030282DD11C
:1062D8002E4A527802F0DF02582A15D02C4A11684B
:1062E80010290DD02D283BD00A2B47D900204BE090
:1062F800012B39D0264A1168102931D12D282BD0ED
:10630800082B3BD900203FE0204A92782D2A09D05B
:106318000A2B2BD810211F48FFF756FF003818BF4B
:10632800012031E00B2BF5D900202DE02528D5D10F
:10633800164A52782D2A09D00B2B19D80A2116484B
:10634800FFF742FF003818BF01201DE00C2BF5D9DC
:10635800002019E00023D1E7092B0FD9002013E012
:106368000B2B0BD900200FE000200DE000200BE0E4
:10637800002009E0064B19681029EBD00348FFF705
:1063880023FF003818BF012008BD00BFE4750020B6
:0C63980080760020E6750020E5750020EE
:1063A40070B41B4D00241B4E06F1FF3C284610F828
:1063B400013B1CF8012FA3F16101C9B219290BD8C3
:1063C400203BDBB2A2F16101C9B219290CD8203AF1
:1063D400D2B29A42EBD014E0A2F16101C9B21929F8
:1063E4000BD9202B08BF002393420AD1002ADED107
:1063F400094B1C60012070BC7047203AD2B2202B9C
:10640400E7D101340835AA2CCED10020F3E700BF30
:0C641400C4A50008E4750020C476002038
:106420001D4B1B788BB330B51B4A00231C46013330
:1064300012F8181F0029F9D1B4F1FF3F27D004EB5F
:106440004405154B03EBC505013D08E0134B1C60EB
:10645000012030BD013C183DB4F1FF3F19D0104977
:1064600001F1100EAC461CF8010F11F8013BA3F12D
:106470006102D2B2192A9CBF203BDBB28342E9D130
:106480000028E3D07145EED1E4E7002070470020FA
:10649000DFE70020DDE700BFBC320020C47600202B
:0464A000E47500207F
:1064A40008B52A4B1A682A4B1A60FFF757FEFFF704
:1064B400B5FF00283ED0254B1A68254B1A60254BA2
:1064C4001B68062B3CD9244A1360244903EB43027E
:1064D400D00001EBC2024FF0000C01F800C0526979
:1064E400C2F30B021E4802601E48026003EB430322
:1064F40001EBC30301F57C618B420AD20139C91A4D
:1065040021F0030104311944604643F8040B8B4223
:10651400FBD140F6FE339A420BD89300043B124A57
:10652400134402F53F523832002143F8041F9342CA
:10653400FBD108BD0D4A136843F021031360F8E74B
:106544000A4A136843F080031360F2E77076002070
:1065540068760020C4760020DC760020BC3200205F
:106564000C77002008770020BC020020FC76002075
:1065740008B50E4B1A680E4B1A60FFF7EFFDFFF7D4
:106584004DFF28B10B4B1B6801330B4A136008BD48
:106594000A4B1B78302B05D0094A136843F02103BA
:1065A4001360F4E7044B00221A60F0E770760020D1
:1065B40068760020C47600201C770020E475002053
:0465C400FC76002041
:1065C800084A1368084941F823000133136040F66C
:1065D800FE32934204D9054A136843F0200313603E
:1065E800704700BF0C770020BC020020FC7600201A
:1065F80008B5154B1868154B53F8203013F4002FC5
:106608000AD1134A12689AB913F4003F0AD1114B00
:1066180053F82030984704E00F4A136843F4007396
:10662800136008BD0C4A136843F008031360F8E7C9
:1066380013F4803F04D0074B53F820309847F0E715
:10664800FFF7BEFFEDE700BFC47600201CA30008DB
:0C6658000077002000000020FC760020ED
:10666400F0B595B00CAC3D4D0FCD0FC495E80F00BF
:1066740084E80F0005AC3A4D0FCD0FC495E8070030
:1066840003C422706C46374D0FCD0FC42B682370A2
:10669400354B1B68522B0DD9344D334FA5F15106A0
:1066A4002C4615F8010FF9F7EDFF0234A41B3B68E3
:1066B400A342F5D852232E4A13602E4A13602C4C61
:1066C4002D4E02E022682B4B1A60274D22682B685E
:1066D4009A4231D2FFF742FD3378002BF6D0FFF710
:1066E400E9FD58B1254B1A68254B1A60254B1B68E8
:1066F400002BE7D0244B01221A60E3E7FFF750FE9A
:1067040080B1224B1A68224B53F8223013F4802FA5
:106714001FD0FFF76FFF1F4B1B683BB92268154B57
:106724001A60D2E70CA804F0B4FD05E0194B00226E
:106734001A60684604F0ADFD0D20F9F7A3FF52235B
:10674400094A13600A4A1360134B00221A6015B0F9
:10675400F0BD05A804F09DFDEEE700BF4CB10008B4
:106764006CB1000888B1000874760020917500208F
:106774007076002068760020E47500206C76002096
:1067840010770020F876002014770020C4760020CB
:0C6794001CA30008FC7600200477002005
:1067A00010B5294B1A68294B1A60FFF7D9FCFFF77F
:1067B00037FE00282DD0244B1A68244B1A60244B36
:1067C0001B6803EB4301234A02EBC102526912F03A
:1067D000404F24D0204A126862B1204A12684AB160
:1067E0001E4A002111601E490A68101D08601D49DB
:1067F000096851601C4A1268BAB91948026852F80F
:10680000044903EB4303134901EBC3031C6102601A
:1068100004E0164A136843F0A003136010BD134A46
:10682000136843F080031360F8E78220FFF7CCFE83
:10683000074B186800EB4000064B03EBC00010301C
:10684000FFF7C2FEEAE700BF7076002068760020FE
:10685000C4760020BC320020F87600201477002097
:10686000B87600201077002000770020FC7600200A
:1068700008B58320FFF7A8FE054A1368191D1160AB
:10688000044A12685A604FF0FF30FFF79DFE08BDC2
:08689000B87600200C7700200F
:1068980008B58420FFF794FE054A1368191D116096
:1068A800044A12685A604FF0FF30FFF789FE08BDAE
:0868B800B87600200C770020E7
:1068C00008B58520FFF780FE054A1368191D116081
:1068D000044A12685A604FF0FF30FFF775FE08BD9A
:0868E000B87600200C770020BF
:1068E80008B58620FFF76CFE054A1368191D11606C
:1068F800044A12685A604FF0FF30FFF761FE08BD86
:08690800B87600200C77002096
:1069100038B58720FFF758FE094C25684FF0FF3047
:10692000FFF752FE074B1A6810680749236803F106
:106930008043013B01EB830341F82030156038BDF3
:0C6940000C770020B8760020BC0200207C
:10694C0008B58820FFF73AFE054A1368191D116037
:10695C00044A12685A604FF0FF30FFF72FFE08BD53
:08696C00B87600200C77002032
:1069740008B58C20FFF726FE054A1368191D11601F
:10698400044A12685A604FF0FF30FFF71BFE08BD3F
:08699400B87600200C7700200A
:10699C0038B58D20FFF712FE0C4C236818680C4D8F
:1069AC0005EB8000FFF70AFE23681A68094B1B6889
:1069BC0003F18043013B05EB830345F822308F2024
:1069CC00FFF7FCFD2368043B236038BDB87600203C
:0869DC00BC0200200C77002032
:1069E40008B5234B1B68BBB9224B1B681968224AA4
:1069F4001160224A934230D9214A1268022A1FD0D8
:106A0400043B1C4A13601F4A1368013B13601E4B6E
:106A14001A681E4B1A6008BD7D20FFF7D3FD0022C3
:106A2400134B1A601A490B6801330B6003EB4303E1
:106A3400DB001849CA54184B1A68184B1A60E6E769
:106A4400104A1168164A12689142D9D1144A002199
:106A540011600B4A03211160D2E7074B00221A6030
:106A6400074B1B68022BD2D1054B03221A60CEE7D9
:106A740000770020C0760020EC76002040730020D0
:106A8400A8020020E0760020D8760020807600203E
:106A9400DC760020BC3200200C7700200877002030
:046AA400187700203F
:106AA80038B5324B1B684BBB314B1B681C6824F450
:106AB8000024A4F17803022B16D97D20F9F7E0FD14
:106AC8002020F9F7DDFDFDF7EBFEA4F18805072D81
:106AD80015D98C3C012C1CD9032D0FD8254B1B68CC
:106AE800188804F0FAFB09E0234B18680430C0F357
:106AF8000B0004F0F2FB2920F9F7C2FD38BD202075
:106B0800F9F7BEFD5220F9F7BBFD3A20F9F7B8FDB9
:106B1800DFE7184B1A68194BD31A082BEED932F84D
:106B28000C0C04F0DAFB2020F9F7AAFD2020F9F775
:106B3800A7FD104C236833F8080C04F0CEFB202086
:106B4800F9F79EFD6920F9F79BFD236833F8040CDB
:106B580004F0C3FB2020F9F793FD7820F9F790FDA6
:106B680023681888043004F0B8FBC7E7FC760020D7
:106B7800E8760020C0760020EC76002040730020E4
:106B880070B5464B002103F57C6243F8041B934221
:106B9800FBD1434B03F54051002243F8042F8B42AD
:106BA800FBD100233F4A13600A223F490A603F494C
:106BB8000A603F4A012111603E4A13603E4A136051
:106BC8003E4A13603E4A13603E4A082111603E4A1D
:106BD800322111603D4A13603D4A13603D4A1360FB
:106BE8003D4A13603D4A13603D4A13602B4B3122E6
:106BF8004FF0560C00214FF0404083F800C05A7007
:106C080099705861196118330132D2B2352AF4D11A
:106C1800224B4E2583F86050532483F861404FF08F
:106C2800540E83F862E04FF0500C83F863C03122B1
:106C380083F86420002283F865204FF040405867AD
:106C48004FF0FF31196783F8785083F8794083F85B
:106C58007AE083F87BC0322683F87C6083F87D2055
:106C6800C3F88C00C3F8881083F8905083F89140DB
:106C780083F892E083F893C0332483F8944083F830
:106C88009520C3F8A400C3F8A010164B072119607B
:106C9800154B1A60FDF7F8FA70BD00BFBC32002032
:106CA800B802002090770020D87600208076002057
:106CB800A80200201C7700209C77002098770020ED
:106CC800A0760020A8760020A4760020F476002084
:106CD800D4760020D0760020F0760020CC760020F4
:0C6CE800C8760020DC7600200C7700202D
:106CF400204B1868D0B9204B1B685BB11F4B1B6835
:106D04001F4A1268934205D032BFD01A981A00F570
:106D1400007070471B4B1B681B4A1268934227D0B4
:106D240032BFD01A981A00F500707047022810D0AC
:106D340004280ED0104B1868D0B1104B1868104BB3
:106D44001B68984213D032BF181AC01A00F500709D
:106D540070470C4B18680C4B1B68984205D032BF27
:106D6400181AC01A00F50070704700207047002000
:106D7400704700BF887700205C76002048770020A9
:0C6D84004C770020787700207C770020FE
:106D900010B5084B1C68221D1A60074B1B682BB1ED
:106DA000064B1B6813B1064B186801E0FFF7A2FF02
:106DB000606010BDB8760020A8020020F8760020A0
:046DC0007C760020BD
:106DC40010B40D4B1C680D4921440D48002311F8E3
:106DD400012F222A04D000F8012B01334E2BF6D1C7
:106DE400074A2221D15401330021D1542344054AB6
:106DF4001360012010BC7047687600203F750020A6
:086E0400E47500207076002007
:106E0C001A4B03445B78A3F16102192A03D8203B87
:106E1C00A3F1370205E02F2B1BD9A3F13002092A6D
:106E2C00F6D80F2A18D8114B18448378A3F16101B6
:106E3C00192907D8203BA3F137000F2812D800EBF3
:106E4C00021070472F2B0AD9A3F130000928F4D96E
:106E5C00F1E74FF0FF3070474FF0FF3070474FF0C5
:106E6C00FF3070474FF0FF30704700BFE4750020D3
:106E7C002DE9F84307464D4B1B6801334C4A136010
:106E8C00FFF79AFF4B4A0026344603E001360134E3
:106E9C00502C0DD012F8013B5C2BF7D0222BF6D1E5
:106EAC00444B00221A55444B1D6845B9414C5DE0DA
:106EBC00424A136843F002031360BDE8F883012FC4
:106ECC000CBF7E207F20FFF779FB3D4A1368A4EBB3
:106EDC0046043C4941F823400133136000263446F4
:106EEC003546344F9046894602E001357B5D6BB3E5
:106EFC007B5D5C2B0ED0A3401E430834182CF4D9B8
:106F0C00D8F8003049F823600133C8F80030002667
:106F1C003446EAE72846FFF773FFB0F1FF3F0FD086
:106F2C000335A04006430834182CDFD9D8F80030BC
:106F3C0049F823600133C8F8003000263446D5E701
:106F4C001E4A136843F002031360B6E7002CB4D05A
:106F5C001B4A13681B4941F8236001331360ACE7EB
:106F6C00F9F78CFB0135635D002BA6D0605D5C28C6
:106F7C0004D0012FF4D0F9F7DBFCF3E72846FFF738
:106F8C003FFFB0F1FF3F06D00335012F09D0C0B24F
:106F9C00F9F7CEFCE7E7094A136843F002031360E4
:106FAC008BE7C0B2F9F76AFBDDE700BF7076002013
:106FBC0068760020E475002000770020FC76002025
:086FCC000C770020BC0200203C
:106FD40008B50E4B1B68032B04D00C4B1B68042B09
:106FE40008D008BDFAF716FE0028F6D0C0B2FAF7AA
:106FF40055FEF2E7064B1B68002BF2D0FBF726FD8B
:107004000028EED0C0B2FAF749FEEAE788770020FC
:047014005C76002086
:1070180008B5314B1B68012B0BD0022B1ED0032B5C
:1070280039D0042B33D02D4A136843F04003136042
:1070380008BD2B4B19680A1D1A602A4B1B682A4A7F
:107048001268934207D0934232BFD31A9B1A03F5B2
:1070580000734B60ECE700234B60E9E7234B1B68A8
:10706800002BE0D01E4B19680A1D1A60204B1B68C4
:10707800204A1268934207D0934232BFD31A9B1A10
:1070880003F500734B60D3E700234B60D0E7174B41
:107098001B68002BC7D0FFF799FFFFF797FFFFF793
:1070A80095FF0F4B1A68111D1960134B1968134B84
:1070B8001B68994204D0994205D25B1A5360B7E71E
:1070C80000235360B4E70A4B1B680A4909685B1A36
:1070D800C3F180035360ABE788770020FC7600207B
:1070E800B8760020787700207C7700205C76002036
:1070F800487700204C770020987700209C77002064
:10710800374B1B68B3F5803F35D3354B4FF6FF72CD
:107118001A60344B1B6813F0010F12D1314B002257
:107128001A611A6030498A6D42F002028A6546F295
:1071380060029A614FF4FA62DA621A6842F0010258
:107148001A60274B1B68013B264A9362274B1B6832
:10715800002B40DB234A136A43F001031362244BDC
:107168001B68002B1F4A136AB4BF23F0100343F0B7
:10717800100313627047002BCBD11A4A136823F00F
:10718800010313604FF0FF30184B18604FF0904325
:10719800196821F440511960D96821F44051D96027
:1071A800D96841F40051D960116A21F001011162D6
:1071B8000F490860196821F440411960D96821F421
:1071C8004041D960D96841F40041D960136A23F07D
:1071D800100313627047136A23F001031362BEE7BA
:1071E800F47600200004004000100240D47600200D
:0471F800D07600202D
:1071FC004FF09042136823F440531360224A136AF1
:10720C0023F001031362214B1B68002B20DB4FF092
:10721C009041CA6822F44052CA6003B3B3F5FA6FC6
:10722C0025DA4FF090431A6842F400521A601A6A39
:10723C0022F070621A621A6A42F000721A62124BE1
:10724C001A6A42F001021A62104A12685A637047B5
:10725C004FF09042D36843F40053D36070470A68F0
:10726C0042F480520A604FF480028A617047074BE7
:10727C004FF4FA621A604FF090431A6842F480524D
:10728C001A6040229A61704700040040D4760020B6
:10729C0008B5124B1B6863B1114B1B684BB1104BFB
:1072AC0000221A600F4A1368191D11600E4A1268E9
:1072BC005A600C4A136853F804090C4908601360AF
:1072CC000B4B1B6813F0010F02D0FFF791FF08BDA9
:1072DC00084B18221A60FFF711FFF6E7F87600202A
:1072EC0014770020B876002010770020D476002088
:0872FC0000040040F4760020BC
:107304004FF09042136823F440431360224A136AF7
:1073140023F010031362214B1B68002B20DB4FF07A
:107324009041CA6822F44042CA6003B3B3F5FA6FCD
:1073340025DA4FF090431A6842F400421A601A6A40
:1073440022F070421A621A6A42F000521A62124B18
:107354001A6A42F010021A62104A12689A6370475D
:107364004FF09042D36843F40043D36070470A68F7
:1073740042F480420A604FF400028A617047074B6E
:107384004FF4FA621A604FF090431A6842F4804254
:107394001A6080229A61704700040040D076002071
:1073A40008B50F4B1B6863B10E4B1B684BB10D4BFB
:1073B40000221A600C4A1368191D11600B4A1268E6
:1073C4005A60094A136853F80409094908601360AC
:1073D400FFF798FEFFF710FFFFF792FF08BD00BF0D
:1073E400F876002014770020B8760020107700206B
:0473F400F47600200B
:1073F80008B5124B1B6863B1114B1B684BB1104B9E
:1074080000221A600F4A1368191D11600E4A12688B
:107418005A600C4A136853F804090C490860136051
:107428000B4B1B6813F0010F02D0FFF767FF08BD75
:10743800084B18221A60FFF763FEF6E7F87600207B
:1074480014770020B876002010770020D07600202E
:0874580000040040F47600205E
:107460003C4B1B68B3F5803F3AD33A4B4FF6FF7263
:107470001A604FF080431B6813F0010F13D14FF0D7
:10748000804300221A611A6033498A6D42F001027A
:107490008A6546F260029A614FF4FA62DA621A680B
:1074A00042F001021A602B4B1B68013B4FF08042F7
:1074B00093622A4B1B68002B44DB4FF08042136A17
:1074C00043F010031362264B1B68002B4FF08042E1
:1074D000136AB4BF23F0010343F001031362704742
:1074E000002BC6D14FF080431A6822F001021A60C7
:1074F0004FF0FF30194A10601A4A116821F0C0019C
:107500001160D16821F0C001D160D16841F08001E3
:10751000D1601A6A22F010021A62114A10604FF00C
:107520009042116821F440611160D16821F44061FA
:10753000D160D16841F40061D1601A6A22F0010281
:107540001A62704702F58062136A23F01003136217
:10755000B9E700BFF076002000100240CC76002092
:08756000C87600200004004879
:10756800244A136823F0C00313604FF08042136A63
:1075780023F010031362204B1B68002B1FDB1D49EF
:10758800CA6822F0C002CA60FBB1B3F5FA6F24DA08
:10759800184B1A6842F080021A601A6A22F4704284
:1075A8001A621A6A42F480521A624FF080431A6AC9
:1075B80042F010021A62104A12689A6370470D4A24
:1075C800D36843F08003D36070470A6842F04002F2
:1075D8000A604FF400228A617047074B4FF4FA6241
:1075E8001A60044B1A6842F040021A6008229A6135
:0C75F800704700BF00040048CC76002063
:1076040008B5134B1B6863B1124B1B684BB1114B8C
:1076140000221A60104A1368191D11600F4A12687B
:107624005A600D4A136853F804090D490860136041
:107634004FF080431B6813F0010F02D0FFF792FF55
:1076440008BD084B18221A60FFF708FFF6E700BFD1
:10765400F876002014770020B876002010770020F8
:08766400CC760020F076002036
:10766C004FF09042136823F4406313604FF0804254
:10767C00136A23F001031362204B1B68002B21DBE0
:10768C004FF09041CA6822F44062CA600BB3B3F564
:10769C00FA6F26DA4FF090431A6842F400621A60CF
:1076AC001A6A22F470021A621A6A42F480121A627E
:1076BC004FF080431A6A42F001021A620F4A1268B4
:1076CC005A6370474FF09042D36843F40063D36021
:1076DC0070470A6842F480620A604FF400128A61B3
:1076EC007047064B4FF4FA621A604FF090431A68D9
:1076FC0042F480621A6020229A617047C87600209A
:10770C0008B50F4B1B6863B10E4B1B684BB10D4B8F
:10771C0000221A600C4A1368191D11600B4A12687A
:10772C005A60094A136853F8040909490860136040
:10773C00FFF790FEFFF712FFFFF792FF08BD00BFA7
:10774C00F876002014770020B876002010770020FF
:04775C00F0760020A3
:1077600008B5134B1B6863B1124B1B684BB1114B2F
:1077700000221A60104A1368191D11600F4A12681E
:107780005A600D4A136853F804090D4908601360E4
:107790004FF080431B6813F0010F02D0FFF766FF24
:1077A00008BD084B18221A60FFF75AFEF6E700BF23
:1077B000F876002014770020B8760020107700209B
:0877C000C8760020F0760020DD
:1077C800104A136853F80409136018280AD9A0F15D
:1077D800A003182B04D90C4A136843F48063136080
:1077E80000F01F000F280BD830F0020303D0A0F1DF
:1077F8000903032B04D8044A136843F48063136015
:0C780800704700BFB8760020FC7600201E
:1078140008B5FFF7D7FF0C4B1B6883B9430003F08F
:107824001E030F2894BF4FF09042084A1269134078
:1078340007490A68101D086013B10123536008BD8D
:1078440000235360FBE700BFFC76002000040048DF
:04785400B8760020E2
:10785800042818D005282CD11E4A136823F4803335
:1078680013601D4B1B68B3F1FF3F0BD0052809D1EE
:107878004FF08042136A23F010031362164B4FF047
:10788800FF321A607047134A136823F0010313602C
:10789800124B1B68B3F1FF3FE3D00728E1D1104A30
:1078A800136A23F0100313620C4B4FF0FF321A6077
:1078B80070470C4B1B68B3F1FF3FE9D00628E7D1AE
:1078C800074A136A23F001031362064B4FF0FF3295
:1078D8001A60704700080050C8760020D076002053
:0878E80000040040D4760020EA
:1078F00070B5FFF769FF244B1B680BBB04464300C0
:1079000003F01E060325B540ED430F2819D91038A2
:10791000162C29D01D4B1B68B3F1FF3F01D0032863
:1079200027D01B4AD3682B40D36013681D401560D5
:107930001468012101FA06F3234313608140916129
:1079400070BDFFF789FF4FF09042D3682B40D360A2
:1079500013681D4015601068012101FA06F3034306
:107960001360A1409161EBE7074B4FF480621A600E
:10797000E6E74FF08042136A23F010031362034BD3
:107980004FF0FF321A60CCE7FC760020CC76002066
:0479900000040048A7
:1079940070B5FFF717FF254B1B6813BB0446450062
:1079A40005F01E050326AE40F6430F281AD9A0F1B0
:1079B400100216282AD01E4B1B68B3F1FF3F01D0DA
:1079C400032A28D01B4BDA683240DA601A68164062
:1079D4001E601A68012000FA05F515431D60A040D9
:1079E400986170BDFFF736FF4FF09043DA6832407C
:1079F400DA601A6816401E601968012202FA05F559
:107A04000D431D601034A2409A61EAE7074B4FF41E
:107A140080621A60E5E74FF08042136A23F0100396
:107A24001362034B4FF0FF321A60CBE7FC76002061
:087A3400CC760020000400489C
:107A3C0038B5FFF7C3FE224B1B68FBB9450005F0B8
:107A4C001E050324AC40E4430F2818D9A0F1100202
:107A5C00162825D01B4B1B68B3F1FF3F01D0032A1E
:107A6C0023D0194B1A6822401A60DA681440DC6083
:107A7C00D968012202FA05F50D43DD6038BDFFF728
:107A8C00E5FE4FF090431A6822401A60DA68144001
:107A9C00DC60D968012202FA05F50D43DD60EDE7E3
:107AAC00074B4FF480621A60E8E74FF08042136A8C
:107ABC0023F010031362034B4FF0FF321A60D0E730
:0C7ACC00FC760020CC760020000400486E
:107AD80038B5FFF775FE224B1B68FBB9450005F06A
:107AE8001E050324AC40E4430F2818D9A0F1100266
:107AF800162825D01B4B1B68B3F1FF3F01D0032A82
:107B080023D0194B1A6822401A60DA681440DC60E6
:107B1800D968022202FA05F50D43DD6038BDFFF78A
:107B280097FE4FF090431A6822401A60DA681440B2
:107B3800DC60D968022202FA05F50D43DD60EDE745
:107B4800074B4FF480621A60E8E74FF08042136AEF
:107B580023F010031362034B4FF0FF321A60D0E793
:0C7B6800FC760020CC76002000040048D1
:107B740010B5FFF727FE1C4B1B68CBB9440004F07B
:107B84001E0303249C40E4430F2812D9A0F11002E1
:107B9400162819D0154B1B68B3F1FF3F01D0032AF7
:107BA40017D0134B1A6822401A60DA681440DC605C
:107BB40010BDFFF74FFE4FF090431A6822401A6041
:107BC400DA681440DC60F3E7074B4FF480621A6014
:107BD400EEE74FF08042136A23F010031362034B65
:107BE4004FF0FF321A60DCE7FC760020CC760020F0
:047BF4000004004841
:107BF80038B5414BDB6C13F4005F00D038BD3E4B09
:107C0800DA6A22F40052DA62DA6C42F40052DA6478
:107C18004FF0A044A36823F00053A360A36843F087
:107C28008053A360354DAB6823F00053AB60AB685D
:107C380043F08053AB600220F9F712F8D4F8B03063
:107C480023F47F4323F0FE03C4F8B030D5F8B030F6
:107C580023F47F4323F0FE03C5F8B030284B4FF4DC
:107C680040329A60F8F71EFC236843F00103236052
:107C7800A36843F00103A3602246136813F0010FC1
:107C8800FBD04FF0A0431A6842F001021A604FF08F
:107C98000042DA601B4A5A6102F160429A6103F5B8
:107CA80080731A6842F001021A609A6842F0010271
:107CB8009A601A46136813F0010FFBD00F4B1A682D
:107CC80042F001021A604FF00042DA600D4A5A6130
:107CD80002F160429A614FF0A04100220A634A63B0
:107CE8008A63CA631A635A639A63DA63F8F7DAFB3A
:107CF800F8F7D8FB82E700BF0010024000010050EF
:087D08000003005024499224FD
:107D10004FF0A0431A6842F001021A609A6842F0DC
:107D200002029A6003F580731A6842F001021A6039
:107D30009A6842F002029A604FF0A042936813F0F2
:107D4000010FFBD1044BDA6C22F40052DA64DA6AD8
:0C7D500042F40052DA627047001002405A
:107D5C0070B588B0874B0DF1100C0FCBACE8070059
:107D6C00ACF80030844BEC460FCBACE807008CF839
:107D7C000030824B1B681C68B4F1FF3F26D0B02C3E
:107D8C0000F0E880082C03D9A4F1A003072B26D817
:107D9C0004F00F056B0003269E40794BDB6C13F44B
:107DAC00005F00F0E0804FF0A04340F2FF721A60D9
:107DBC006B1E072B00F2A780DFE813F01700A5005D
:107DCC0039004400540073008C00C100043B6B4A22
:107DDC001360FFF797FF684603F057FA25E0694AEE
:107DEC00136843F4806313601FE04FF090431A68EC
:107DFC0032431A60DA6822EA0606DE60022314F0C7
:107E0C000C0F40F086809B014FF0A04213639368E7
:107E1C0043F004039360136813F0080FFBD0574B27
:107E2C001B684FF0A042126C1A6008B070BD4FF086
:107E3C0090431A6832431A60DA6822EA0606DE605A
:107E4C000423DCE7504A136823F0010313604FF05E
:107E5C0090431A6832431A60DA6822EA0606DE603A
:107E6C001123CCE7494B1B68B3F1FF3F09D04FF00E
:107E7C008042136A23F001031362444B4FF0FF322C
:107E8C001A60414A136823F4803313604FF0904317
:107E9C001A6832431A60DA6822EA0606DE600D239D
:107EAC00ADE73B4B1B68B3F1FF3F08D0394A136A6F
:107EBC0023F001031362364B4FF0FF321A604FF080
:107ECC0090431A6832431A60DA6822EA0606DE60CA
:107EDC00032394E7304B1B68B3F1FF3F08D02D4AC6
:107EEC00136A23F0100313622B4B4FF0FF321A600E
:107EFC004FF090431A6832431A60DA6822EA060699
:107F0C00DE6004237BE71F4A136843F4806313602D
:107F1C008BE79B01214A1363936843F0040393603E
:107F2C00136813F0080FFBD0144B1B681B4A126C20
:107F3C001A607AE74FF0A04340F2FF721A60184BB8
:107F4C001A6842F003021A60DA6822F00302DA605F
:107F5C000F2358E70A4BDB6C13F4005FEAD14FF4A4
:107F6C00403608252C46FFF741FE04A803F08DF996
:107F7C0019E700BF9CB10008ACB10008B87600202E
:107F8C0000100240FC76002000080050C87600204B
:107F9C00D476002000040040D07600200001005070
:047FAC000004004885
:107FB000174B1B68032B24D8164B1B68043B1C2B48
:107FC0001FD8154B1B68B3F5803F1AD2134B1A68A4
:107FD00022F47C621A601A6842F488621A60DA68D5
:107FE00022F44072DA60DA6842F40072DA60084B18
:107FF0001B68012B094B8CBF08224FF400229A61A9
:108000007047074A136843F480631360704700BFEA
:10801000A0760020A8760020A47600200004004866
:04802000FC760020CA
:1080240010B50C4A1368194651F804490A4804600B
:10803400116053F8040C09490860A3F108011160A8
:1080440053F8080C064908600C3B1360FFF7AEFFB9
:1080540010BD00BFB8760020A4760020A8760020CA
:04806400A0760020E2
:108068002DE9F0479E4B1B6803F4A863B3F5886FAE
:108078002BD19C4B1B681D689B4B1A689B4B1C683B
:10808800002C5BD1964B4FF400219961984B1868EE
:10809800F0B90127924B4FF4001E4FF0200C0E460A
:1080A8000824013A07FA02F1294214BFC3F818C09C
:1080B800C3F818E09E611969C1F3001141EA400054
:1080C8009C61002AEDD104462FE0FFF76DFFD0E751
:1080D8004FF00108824E4FF4001A4FF020094FF478
:1080E800002E834F83484AF6AA214FF0080C013A24
:1080F80008FA02F32B4214BFC6F81890C6F818A065
:10810800C6F818E03B6813B10160013BFCD1336944
:10811800C3F3001343EA4404C6F818C03B6813B11C
:108128000160013BFCD1002AE1D16D4B4FF40022E4
:108138009A616C4B1B681C60BDE8F087012C25D048
:10814800022C78D0664B08219961694B1C68002C79
:1081580040F0D2800127624B4FF4001E4FF0200CF4
:108168004FF400260846013A07FA02F1294214BFE3
:10817800C3F818C0C3F818E09E611969C1F300116B
:1081880041EA44049861002AEDD1E3E0544B4FF4EE
:1081980000219961564B1C68D4B90127504B4FF404
:1081A800001E4FF0200C08260846013A07FA02F193
:1081B800294214BFC3F818C0C3F818E09E611969B2
:1081C800C1F3001141EA44049861002AEDD12DE081
:1081D80000244FF00108424E4FF4001A4FF02009D6
:1081E8004FF0080E424F43484AF6AA214FF4002C9C
:1081F800013A08FA02F32B4214BFC6F81890C6F8E1
:1082080018A0C6F818E03B6813B10160013BFCD127
:108218003369C3F3001343EA4404C6F818C03B6843
:1082280013B10160013BFCD1002AE1D12C4B4FF482
:1082380000229A617DE72A4B082199612C4B1C6822
:10824800DCB90127264B4FF4001E4FF0200C0E46D8
:108258004FF40020013A07FA02F1294214BFC3F88B
:1082680018C0C3F818E09E611969C1F3001141EA0A
:1082780044049861002AEDD12DE000244FF0010854
:10828800174E4FF4001A4FF020094FF0080E184F00
:1082980018484AF6AA214FF4002C013A08FA02F3CA
:1082A8002B4214BFC6F81890C6F818A0C6F818E0F4
:1082B8003B6813B10160013BFCD13369C3F3001380
:1082C80043EA4404C6F818C03B6813B10160013B97
:1082D800FCD1002AE1D1024B08229A6129E700BFAC
:1082E80000040048B8760020A8760020A076002078
:1082F800A47600200030004000244FF00108174EFB
:108308004FF4001A4FF020094FF4002E144F15486F
:108318004AF6AA214FF0080C013A08FA02F32B4258
:1083280014BFC6F81890C6F818A0C6F818E03B683D
:1083380013B10160013BFCD13369C3F3001343EA75
:108348004404C6F818C03B6813B10160013BFCD176
:10835800002AE1D1014B08229A61EAE600040048AC
:08836800A47600200030004063
:10837000304B1B6F002B5BDD2F4A1268002A2CDB71
:108380002E490A602E4A1268032A4AD8DFE802F012
:10839000020F14194FF090424FF4003191614FF4E5
:1083A0008011916126490A6801320A6011E04FF09C
:1083B000904210219161F5E74FF0904202219161C6
:1083C000F0E74FF090424FF4801191611C4A002178
:1083D0001160013B174A13677047524217490A6000
:1083E000174A1268032A1CD8DFE802F0020B1015A6
:1083F0004FF090424FF4003191614FF48011916140
:10840000D0E74FF0904202219161CBE74FF09042CC
:1084100010219161C6E74FF090424FF40031916115
:10842000D4E707490A6801320A60032ACEDCD0E7A4
:10843000704700BFBC32002090760020B476002048
:048440009C76002006
:1084440008B5384B1B6863B1374B1B684BB1364BCF
:1084540000221A60354A1368191D1160344A1268E3
:108464005A60344B1B6FB3F1FF3F29D0324B1B686A
:108474006BB9324A1360324A13604FF090431A6862
:1084840022F443721A601A6842F482721A6027490D
:108494000B6853F80429284802600B6052B94FF066
:1084A40090434FF400329A614FF480129A61214B49
:1084B40000221A67224B00221A60FFF757FF08BDFB
:1084C4001D4B00221A604FF090431A6822F4437245
:1084D4001A601A6842F482721A60144B1A6813689C
:1084E400002B09DD4FF090434FF400329A611022C3
:1084F4009A61FEF7D1FEE2E7002B08DB4FF09043D0
:108504004FF400329A614FF480129A61F1E75B42B2
:1085140013604FF0904302229A614FF480129A61E3
:10852400E7E700BFF876002014770020B876002033
:1085340010770020BC320020907600209C7600202A
:04854400B4760020E9
:108548002E4BD3F88830002B56DD2D4A1268002AAE
:108558002ADB2C490A602C4A1268032A45D8DFE82E
:1085680002F00212171B294A4FF4000191614FF0E3
:108578008071916124490A6801320A60013B1F4AEF
:10858800C2F888307047214A4FF480719161F1E751
:108598001E4A80219161EDE71C4A4FF0807191617C
:1085A800194A00211160E9E7524216490A60164A41
:1085B8001268032A19D8DFE802F0020A0E13134AD8
:1085C8004FF4000191614FF080719161D2E70F4A39
:1085D80080219161CEE70D4A4FF480719161C9E71E
:1085E8000A4A4FF400019161DAE707490A68013243
:1085F8000A60042AD4D0C1E7704700BFBC3200200B
:108608008C760020B0760020987600200004004880
:1086180008B5364B1B6863B1354B1B684BB1344BFF
:1086280000221A60334A1368191D1160324A126811
:108638005A60324BD3F88830B3F1FF3F28D0304B23
:108648001B6863B92F4A13602F4A13602F4B1A68AF
:1086580022F470321A601A6842F4A0321A6025496E
:108668000B6853F80429264802600B6052B9274B5F
:108678004FF400029A614FF080729A611F4B0022FA
:10868800C3F88820204B00221A60FFF759FF08BD65
:108698001B4B00221A601D4B1A6822F470321A60B4
:1086A8001A6842F4A0321A60124B1A681368002B39
:1086B80009DD164B4FF400029A614FF480729A61FB
:1086C800FEF796FEE3E7002B07DB104B4FF40002A2
:1086D8009A614FF080729A61F2E75B4213600B4B2C
:1086E80080229A614FF080729A61E9E7F87600205B
:1086F80014770020B876002010770020BC320020C4
:108708008C76002098760020B0760020000400487F
:10871800324BD3F8A030002B5FDD314A1268002AB3
:108728002EDB30490A60304A1268032A4ED8DFE847
:1087380002F00211151B4FF090424FF00041916179
:1087480002F580624FF48011916127490A6801326D
:108758000A6010E0254A10219161F6E74FF0904237
:108768004FF400419161F0E7204A4FF48011916184
:108778001D4A00211160013B184AC2F8A030704719
:10878800524218490A60184A1268032A1ED8DFE8BC
:1087980002F0020D13174FF090424FF00041916123
:1087A80002F580624FF480119161CEE74FF090425C
:1087B8004FF400419161C8E70C4A10219161C4E768
:1087C8004FF090424FF000419161D1E706490A68A5
:1087D80001320A60032ACBDCCDE77047BC320020A7
:1087E80088760020AC7600209476002000040048AB
:1087F80008B5174B1B68022B1DD8164B1B6F2BB1E6
:10880800154B1B6813B1154B1B68BBB1114BD3F843
:1088180088302BB1124B1B6813B1124B1B6883B104
:108828000C4BD3F8A0302BB10F4B1B6813B10F4B77
:108838001B684BB108BDFEF7C9FBDEE7FFF794FDE7
:10884800E4E7FFF77DFEEBE7FFF762FFF2E700BF23
:1088580088770020BC32002090760020B476002073
:108868008C760020B076002088760020AC76002038
:1088780008B50023064A1360064A1360064A1360C7
:10888800FFF7B6FFFDF778FB0028F9D008BD00BF59
:0C88980070760020747600200477002029
:1088A40008B5FFF7A7FF124B1B68022B06D0114B2C
:1088B400186810B1104B186828B908BD0C4B002279
:1088C4001A600120F9E7FDF759FB012807D00228B7
:1088D40008D00A4B1868003818BF0120EDE7FDF7EF
:1088E400BFFEF6E7054A136843F480731360F0E7AC
:1088F40078760020A8020020F8760020FC7600207C
:1089040008B5254B1B68012B0BD0022B19D0032B68
:108914002FD0042B29D0214A136843F0400313605D
:1089240008BDF9F777F9034620B9FFF7B9FF002826
:10893400F7D0F5E71A490A68101D0860DBB25360E6
:10894400EEE7184B1B68002BE5D0FAF77FF80346D7
:1089540020B9FFF7A5FF0028F7D0E1E710490A681E
:10896400101D0860DBB25360DAE70E4B1B68002B66
:10897400D1D0F9F735FA034630B9FEF729FBFFF7F2
:108984008FFF0028F5D0CBE705490A68101D086061
:1089940023F07F435360C3E788770020FC760020F0
:0889A400B87600205C7600208B
:1089AC0010B5084A136853F80409074908601360A6
:1089BC000C4623682BB1F8F789F8FFF76DFF0028F8
:0C89CC00F7D010BDB8760020E476002043
:1089D80008B5054B1A681368642101FB03F313609B
:0C89E800FFF7E0FF08BD00BFB8760020DC
:1089F400F8B51A4A136853F8041C186843F8040CB1
:108A040013681960164D174C05F5007022462B4665
:108A140013F8011F02F8011F8342F9D1124E37687F
:108A240000233360FDF73AF83760104B1B6803B13D
:108A3400F8BD0A4B1A681368642101FB03F3136041
:108A4400FFF7B2FF0A4A0B4914F8013F05F8013F4A
:108A540002F8013F8C42F7D1EAE700BFB876002064
:108A6400336B0020376D002024770020FC76002033
:088A74003B6F0020376F00206A
:108A7C0008B5474B1B6863B1464B1B684BB1454B64
:108A8C0000221A60444A1368191D1160434A126887
:108A9C005A60434BD3F8A030B3F1FF3F36D0414B73
:108AAC001B68BBB9404A1360404A13604FF09043B7
:108ABC001A6822F040421A601A6842F080421A602A
:108ACC0003F580631A6822F440721A601A6842F443
:108ADC0080721A6030490B6853F8042931480260DF
:108AEC000B606AB94FF090434FF000429A6103F566
:108AFC0080634FF480129A61294B0022C3F8A020A6
:108B0C002A4B00221A60FFF701FE08BD254B0022FC
:108B1C001A604FF090431A6822F040421A601A68AB
:108B2C0042F080421A6003F580631A6822F44072A6
:108B3C001A601A6842F480721A60174B1A6813682C
:108B4C00002B0BDD4FF090434FF000429A6103F580
:108B5C00806310229A61FEF74FFDD6E7002B0ADBEB
:108B6C004FF090434FF000429A6103F580634FF44D
:108B7C0080129A61EFE75B4213604FF090434FF421
:108B8C0000429A6103F580634FF480129A61E2E728
:108B9C00F876002014770020B8760020107700209B
:108BAC00BC3200208876002094760020AC76002021
:108BBC0038B50D4C236818680C4D05EB8000FDF79B
:108BCC00FDFC23681A680A4B1B6803F18043013BC8
:108BDC0005EB830345F822308E20FDF7EFFC23686C
:108BEC00043B236038BD00BFB8760020BC020020D7
:048BFC000C770020D2
:108C000038B5A9280AD8174C04EBC00401E0F7F7DF
:108C10003BFD14F8010B0028F9D122E0124B1B6830
:108C200003EB4301114A02EBC1021269904209D0E1
:108C300003EB43020D4901EBC202013B183A1169F3
:108C40008142FAD103EB4303DB00084D5C1E2C4448
:108C50000F351D4414F8010F18B1F7F715FDAC429C
:108C6000F8D138BDC4A50008DC760020BC32002055
:108C70002DE9F04383B0904B93E803000090ADF8EA
:108C800004108E4B1D6815B103B0BDE8F0838C4B0A
:108C90001B688C4A1360D3F8009029F400278A4B94
:108CA0001E6806EB46060D20F7F7EEFC46B12C4693
:108CB0004FF020084046F7F7E7FC0134A642F9D10F
:108CC000804B188802F00DFB2020F7F7DDFC1FFA1F
:108CD00089F002F006FB2020F7F7D6FCAA2F15D862
:108CE0003846FFF78DFF832F45D0842F48D0852F3E
:108CF0006CD0862F72D0872F49D08A2F76D0892FBB
:108D00007AD08D2F43D08B2F41D04DE02D20F7F717
:108D1000BBFC3E20F7F7B8FC2020F7F7B5FC38463F
:108D2000FFF76EFF822F00F088807D2F00F0A0807B
:108D3000664C654E032D00F0AE802368022B40F296
:108D4000AA80F7F7C9FEFDF7D5FF0028F2D0FDF79E
:108D500017F90546012800F09580022800F095805B
:108D60000428E7D13368002B00F09580584A13603F
:108D700002232360DEE7574B1B681B683BB1D1E73A
:108D8000544B1B681A6853F8043C9A42CAD0684690
:108D900002F081FA4A4B1B685868043080B202F036
:108DA000A0FA2920F7F770FC802F31D12820F7F79F
:108DB0006BFC494B1B68102B24D0414B1B68586837
:108DC000F8F724FD2920F7F75FFCAEE7414B1B685D
:108DD00053F8042C1B689A42D9D2A3E73D4B1B6879
:108DE00053F8042C1B689A42D1D99BE7394B1B6876
:108DF0001B68002BCBD195E7364B1B681B68002BFB
:108E0000C5D08FE72E4B1B68586802F0ACFAD9E743
:108E1000812F87D12A4B1B685E68A6F11004282099
:108E2000F7F732FC207820B1F7F72EFC0134A64288
:108E3000F8D12920F7F728FC7AE72820F7F724FC57
:108E40001F4B1B685E68A6F11004207820B1F7F76D
:108E50001BFC0134A642F8D14020F7F715FC184B53
:108E60001B68988802F07FFA2920F7F70DFC5FE76E
:108E70002020F7F709FC3C20F7F706FC2D20F7F738
:108E800003FC55E7FDF7EEFB54E70C4A136843F487
:108E900080731360F8E62020F7F7F6FB783F022F87
:108EA00003D8684602F0F7F9EEE67B20F7F7ECFB13
:108EB0002020F7F7E9FBE7E6E4AE0008FC760020A7
:108EC000EC760020E8760020E0760020A802002062
:0C8ED00018770020B87600208076002083
:108EDC0008B5FFF7C7FE064B1B6843B9054B1B686B
:108EEC001A68054B53F822309847FDF7D7FD08BD9B
:0C8EFC00FC760020EC7600200000002036
:108F080008B51A4A136801331360194B19680A1D0A
:108F18001A60184A13684B601B6823F40023136017
:108F28001B6823F40022A92A0BD8134A1268032AC3
:108F380004D0124A52F82330984708BDFFF7CAFFF9
:108F4800FBE70D4B1B68032B06D00D4B1B68002B52
:108F5800F3D1FFF7D5FFF0E7FFF786FE084B1B6854
:108F6800002BEAD1FDF79CFDEFE700BFE07600207B
:108F7800C0760020EC760020A80200200000002027
:048F8800FC76002053
:108F8C00F0B587B001AC374D0FCD0FC42B682370F3
:108F9C00354B364E06EB8306354B1B68B3425BD222
:108FAC00344D334C344F35E0FBF7F2FB39E0FFF72F
:108FBC00A5FF24E0FDF798FE50B923681B68A92B88
:108FCC0018D82A68032A12D057F82330984716E08D
:108FDC00FCF7D0FF012807D00228EED1274A1368EE
:108FEC0043F48073136037E0FDF736FBE5E7FFF7DA
:108FFC006FFF04E02B68032B1BD0FFF77FFFFFF7FD
:10900C00F5FB1E4B1B683BBB2368BBB104332360D1
:10901C00B34221D22B68002BCCD1194B1B68042BEB
:10902C00C2D023681B68A92BC1D857F823309847A6
:10903C00E5E7FFF717FEFDF731FDDEE70D4B1B688B
:10904C00032B0BD00B4B01221A6000230D4A13602B
:10905C000D4A13600D4A136007B0F0BD01A802F071
:10906C0014F9EFE7BCB100087C420020BC020020E0
:10907C00EC760020A802002000000020FC760020E6
:10908C0078760020F876002014770020E076002017
:10909C00F8B52D4B1C68002C33D12C4B1B6803EB03
:1090AC0043012B4A02EBC102526912F0404F0CD023
:1090BC00284A1168081D106003EB4303244A02EB95
:1090CC00C3031B694B602046F8BD214A02EBC10368
:1090DC001B6923F40023204A1360204B01221A60E1
:1090EC001F4D2F681F4C266852232B6023601E4B8C
:1090FC0000221A60FFF744FF2F6026601B4B1C6890
:10910C00E1E7124B1B6803EB4301114A02EBC1026E
:10911C00546914F0404406D10D4A02EBC10318699E
:10912C00FDF74CFACFE78120FDF748FA074B18689A
:10913C0000EB4000064B03EBC0001030FDF73EFA8D
:10914C000A4B1C68BFE700BF00770020C4760020E4
:10915C00BC320020B8760020EC760020F876002097
:10916C00747600207076002004770020FC760020B6
:10917C0070B50023274A1360274A13601546274E03
:10918C0009E08020FDF71AFA254B1868FDF716FA4E
:10919C002A68204B1A60234C2A6823689A4219D2F9
:1091AC00FCF7D8FF3378002BF6D0FDF77FF858B1D9
:1091BC001D4B1B68002BE4D11C4A1368191D116050
:1091CC00174A12685A60E3E7FDF724F938B1FFF744
:1091DC005FFF00B170BD2A680E4B1A60DBE7FDF72C
:1091EC00DBF848B1FDF702FA114B1B68002BF1D1EB
:1091FC002A68084B1A60CEE70D4A136843F0010346
:10920C0013600C4B1A680C4B1A60034B1A68014B19
:10921C001A60DFE76876002070760020E475002085
:10922C006C7600207476002000770020B876002041
:0C923C00FC760020087700200C77002052
:109248002DE9F04F93B00CACAA4D0FCD0FC495E8A3
:10925800030044F8040B217007ACA74D0FCD0FC4D1
:109268002B6824F8023B1B0C2370A44B03AC0FCBD8
:1092780007C42380A24B1A68A24B1A60FCF76CFF44
:10928800FDF7CAF860B9FDF789F828B99E4A13684E
:1092980043F001031360FCE00CA801F0F8FFF8E0CC
:1092A800974B1A68974B1A6007A801F0F0FF974D83
:1092B800286800EB4000964C04EBC00002F04FF821
:1092C8000D20F7F7DDF92B6803EB430204EBC2042A
:1092D800246914F4002F17D024F400248D48241A8C
:1092E800A40803EB43038A4A02EBC3035B6913F048
:1092F800404840F0D180874B53F824307D2B00F054
:10930800B9800126834D2AE003EB4302804901EB33
:10931800C2025469C4F30B04E3E70D20F7F7B0F970
:1093280046461CE001342820F7F7AAF955F824002E
:10933800043080B202F013F82920F7F7A1F90136BA
:109348002020F7F79DF92020F7F79AF9013455F80E
:1093580024307D2B00F08E800136072EDDD805EBFA
:10936800840080B201F0B9FF3A20F7F789F955F87F
:109378002400FFF741FC55F8243023F40023A3F11F
:1093880083020A2ACED9802B13D0812B27D0822B97
:1093980032D07E2BD4D12220F7F772F9631C55F80E
:1093A80023900234B9F1000F5ED0CDF8048047460F
:1093B80048E001342820F7F763F9574B1B68102B56
:1093C80008D055F82400F8F71DFA2920F7F758F9BE
:1093D8000136B5E755F8240001F0C1FFF5E701347F
:1093E8002820F7F74DF955F8240001F0E0FF29206F
:1093F800F7F746F90136A3E701342820F7F740F9D3
:1094080055F8240001F0D3FF4020F7F739F935F873
:10941800240001F0A4FF2920F7F732F901368FE77D
:109428005C20F7F72DF94FEA1B10F7F7ABFA0AF0B3
:109438000F00F7F7A7FA0837182F88BF4746B9F182
:10944800010911D01FB955F8243001930134019B4B
:1094580023FA07FA5FFA8AFBABF120035E2BDFD809
:109468005846F7F70DF9E6E7013C2220F7F708F927
:10947800033665E7274800EB840080B201F02DFF32
:109488003A20F7F7FDF83B20F7F7FAF80D20F7F741
:10949800F7F813B0BDE8F08F03A801F0F8FE1E4BF3
:1094A8001B68102B1BD0194B1B6803EB4303184A8E
:1094B80002EBC303186901F0FEFB2020F7F7E0F880
:1094C8004020F7F7DDF8114B1B6803EB4303104806
:1094D80000EBC300103080B201F041FFD6E70B4B20
:1094E8001B6803EB43030A4A02EBC303186901F044
:1094F80036FFE2E7F4AE00080CAF000820AF000822
:109508007076002068760020FC760020C476002063
:0C951800BC320020BC0200208076002045
:1095240038B51B4C1B4D2B682360FCF717FE2B68CA
:109534002360194B1B6823B35D1E03EB4303174CD5
:1095440004EBC304193C06E0284638BD013D183C31
:10955400B5F1FF3F18D0124901F1100EA4461CF8D2
:10956400010F11F8013BA3F16102D2B2192A9CBF89
:10957400203BDBB28342E9D10028E5D07145EED12E
:10958400E4E74FF0FF30E0E74FF0FF30DDE700BFE6
:109594006876002070760020DC760020BC32002043
:0495A400E47500204A
:1095A80038B5FFF7BBFFB0F1FF3F0FD0044600EB23
:1095B8004003294A02EBC3035B6913F0404F0BD009
:1095C800264A136843F08003136038BD234A1368A2
:1095D80043F021031360F8E7FFF7A0FFB0F1FF3F66
:1095E80027D000EB40031C4A02EBC3035B6913F06E
:1095F800404F24D1844228D3174B04EB440403EB97
:10960800C404256945F4002500EB400203EBC202BF
:1096180014691561124B134A1268191D01EB820176
:1096280053F8042BA24208BF43F8045C8B42F7D1DD
:10963800CBE70A4A136843F021031360C5E7074ADA
:10964800136843F080031360BFE7044A136843F0CC
:1096580080031360B9E700BFBC320020FC7600200D
:08966800BC020020087700207D
:1096700010B5FFF757FFB0F1FF3F24D000EB4003D8
:10968000174A02EBC30319695B69C3F30B03154C5B
:1096900004EB830421F40023A3421AD900EB400019
:1096A0000F4B03EBC00004610E4B0F4A1268181DEC
:1096B00000EB820053F8042B8A4208BF43F8044CA5
:1096C0008342F7D110BD094A136843F021031360A8
:1096D000F8E7064A136843F080031360F2E700BF1F
:1096E000BC320020BC02002008770020FC7600205D
:1096F0002DE9F041154A13685D6808331360FDB128
:109700000746002490460CE0012F13D026FA04F0FF
:10971000C0B2F7F713F90834192C28BF0024013D13
:109720000ED0002CF0D1D8F8003053F8046BC8F8F4
:109730000030E9E726FA04F0C0B2F6F7A5FFEAE741
:10974000024A1368043B1360BDE8F081EC76002008
:1097500010B58AB00DF10C0C134C0FCCACE80F0017
:1097600094E80700ACE803002CF8022B120C8CF8EC
:1097700000200E4A6B4607CA03C31A8003A801F0F3
:109780008AFDF8F76DFA0028FBD0C3B2592B05D03B
:10979000684601F080FD00200AB010BD0D20F6F7EC
:1097A00073FF0120F8E700BF54AF000870AF000856
:1097B00070B590B00546EC46364C0FCCACE80F00C7
:1097C0000FCCACE80F0094E80F008CE80F00324C8F
:1097D000324E33682360FCF7C3FC33682360FCF728
:1097E0006BFD38B12E4A136843F0800313600020EC
:1097F00010B070BD0446FCF7D5FD30B929490DF114
:10980000300C01F1100E60460DE0684601F043FD9A
:10981000FFF79EFF0028F1D10220E9E710F8013C94
:1098200073B171450CD011F8013B00F8013BA3F175
:109830006102D2B2192AF1D8203B00F8013CF0E7CE
:1098400000238DF83F309DF830307BB1164A116807
:1098500001EB4101154A02EBC102013A02F8013F56
:1098600001341CF8013F0BB10F2CF7D10E4B1B68D4
:109870000E4A03EB430002EBC00004440021617078
:109880000B4909680B4C04EB8104046129434161D5
:109890000120ADE7ECA20008687600207076002079
:1098A000FC760020E4750020DC760020BC3200202D
:0898B0000C770020BC0200202F
:1098B80038B54FF04040FFF777FF78B10A4C0B48B6
:1098C8000368226852F8045903EB430C084901EB7A
:1098D800CC010D6122600133036038BD054A13686D
:1098E80043F001031360F8E7B8760020DC76002027
:0898F800BC320020FC760020C8
:1099000008B50020FFF754FF40B1022807D0084BEC
:109910001A68084B1A60084B01221A6008BD074BF1
:109920001B6803EB4303DB00054A0021D154F5E734
:109930000C7700200877002000770020DC760020DC
:04994000BC32002015
:1099440030B5A3B01AAC414D0FCD0FC495E80F004C
:1099540007C4237012AC3E4D0FCD0FC495E80F0021
:1099640084E80F000DF1240C3A4C0FCCACE80F0046
:109974000FCCACE80F002368ACF800300DF1040CF8
:10998400354C0FCCACE80F0094E80F00ACE80700AE
:109994002CF8023B1B0C8CF80030304B1B681C6805
:1099A400042C21D8043B2D4A13602D4B1B689C4288
:1099B4001FD0022C1FD0042C1DD0012C26D0032C28
:1099C40031D0274B1C60274B1B68274A12689A42E8
:1099D4000FD0254A1360F6F7DDFD1AA801F059FCF3
:1099E4000D20F6F74FFE04E0204A136843F4806329
:1099F400136023B030BD12A801F04BFC0D20F6F724
:109A040041FEFFF7A3FE0028D7D1F2E709A801F031
:109A140040FC0D20F6F736FEFFF798FE0028E8D04C
:109A24000F4B1C60E5E701A801F033FC0D20F6F7AD
:109A340029FEFFF78BFE0028DBD00B4B1F221A6098
:109A4400F6F7A8FD064B03221A60D2E7D0B100084E
:109A5400F0B1000810B2000834B20008B876002053
:109A640088770020B077002080770020FC760020E3
:109A740030B585B01A4B93E803000290ADF80C1092
:109A8400090C8DF80E10174B93E803000090ADF805
:109A94000410090C8DF80610F9F766FC124C2368C3
:109AA4001D6802A801F0F5FBFAF7C8FE2020F6F7BE
:109AB400E9FD23681C68684601F0EBFBFAF7BEFE7B
:109AC4002020F6F7DFFDFFF741FE08B905B030BDF1
:109AD400064B1D60064B1C60F7F7D2F8F6E700BF93
:109AE40054B200085CB20008B87600203877002031
:049AF4009477002043
:109AF80030B583B01F4B93E8030000908DF8041035
:109B08001D4A136853F804491360022C06D91B4AEE
:109B1800136843F48063136003B030BD684601F0F6
:109B2800B6FB174801F0B3FB04F13000C0B2F6F7FA
:109B3800A7FDD4B12020F6F7A3FD3F20F6F7A0FD3E
:109B4800FFF702FE0028E7D00E4D2C60F7F796F8D5
:109B58002B68002BE0D0F7F759F90028DCD1074A29
:109B6800136843F020031360D6E7074801F08FFB22
:109B7800E0E700BF64B20008B8760020FC76002059
:0C9B880088B200089077002074B200083A
:109B940030B583B0274B93E8030000908DF8041090
:109BA400254A136853F804491360022C06D9234A42
:109BB400136843F48063136003B030BD684601F05A
:109BC40068FB1F4801F065FB04F13000C0B2F6F7F2
:109BD40059FD74B12020F6F755FD3F20F6F752FDEC
:109BE400FFF7B4FD0028E7D0164B1C60F6F76AFDBA
:109BF40014E0154801F04DFB2020F6F743FD3F200B
:109C0400F6F740FDFFF7A2FD0028D5D00D4C002546
:109C14002560FCF7B7FFF6F751FC25600B4B1B687A
:109C2400002BC9D004490A68101D08605360FBF773
:109C340035FFC1E76CB20008B8760020FC7600203E
:109C440088B200089077002074B2000834770020AE
:109C540030B42C4A936D43F4003393654FF0904332
:109C64001A6822F010021A601A6842F020021A6080
:109C74009A6822F020029A609A6842F010029A6070
:109C84005A6842F001025A6001229A611A6822F06D
:109C940002021A601A6842F001021A609A6822F0FD
:109CA40002029A609A6842F001029A601A6A22F4E7
:109CB40070621A621A6A42F4E0621A62124BC0229B
:109CC400DA604FF400525A6000229A6009221A6046
:109CD4000E4B5A1E0E4D0F4C0F48104903F5007CD5
:109CE400002302F8013F05F8013F04F8013F00F8A2
:109CF400013F01F8013F6245F3D1094B00221A608C
:109D040030BC704700100240004400403C6F00200B
:109D1400336B00202B670020276500202F6900206B
:049D24003077002074
:109D2800C82303494AF6AA220A60013BFCD17047BE
:049D380000300040B7
:109D3C0010B51924FFF7F2FF631E13F0FF04F9D1DD
:109D4C004FF090434FF480329A611224FFF7E6FFF4
:109D5C00631E13F0FF04F9D14FF0904301229A6176
:109D6C00FFF7DCFFFFF7DAFF054AD36913F0800F2A
:109D7C00FBD00023024A9362024A136010BD00BF5D
:089D8C0000440040287700208C
:109D9400104B195C104B1A5C914219D01FFA81FCCC
:109DA40093B28CBFACEB0303A3EB0C039BB21B027B
:109DB4000A4A1268B3FBF2F3C3F30721084A1154A9
:109DC400084A1354084B00221A54084B01221A6003
:109DD400704700BF3C6F0020346B002024770020C4
:109DE4002C6700202865002030690020207700209F
:109DF40008B50346084A126832B9084A1268084985
:109E040088540849885408BD044A1068044A135405
:109E1400FFF7BEFFF7E700BF24770020307700206C
:089E2400346B00203C6F0020AC
:109E2C002DE9F04F0020204B1860204B591E204F7D
:109E3C00204E214C214D03F2FF1E82464FF00109AA
:109E4C004FF0FF080DE0A2EB0A029342B8BF134695
:109E5C008CF80030CA464046013601340135714554
:109E6C001AD001318C460A7817F8013F9A42F3D088
:109E7C0096F800A0207895F800B058442070FF2880
:109E8C0084BF0AF1010A5FFA8AFA9A42DBD2524481
:109E9C009342A8BF1346DBE7BAF1000F01D0024B87
:109EAC001860BDE8F08F00BF207700203C6F0020C9
:109EBC00336B00202C6700203069002028650020BF
:109ECC004FF0FF0C1CEAD0521EBF1CEAD153FF2AE4
:109EDC00FF2B28D01A444FF0004C90EA010313EAF0
:109EEC000C034CEA01214CEA0020A0FB01C1B1F1AA
:109EFC00004F62F17F0238BF49004CEA416CFE2AE8
:109F0C0009D253EA11204CEAC07C28BFBCF10103F2
:109F1C0040EBC2507047124244BF18467047FF20B6
:109F2C0043EAC050704710EACC5F08BF00F0004015
:109F3C0011EACC5F08BF01F000410CEAD153FF2AB3
:109F4C0018BFFF2B03D0484000F00040704700289A
:109F5C001EBFB0F1004F0029B1F1004F11D0FF2A04
:109F6C0002D15FEA402C0CD1FF2B02D15FEA412CCD
:109F7C0007D1484000F0004040F0FE4040F40000A3
:0C9F8C0070474FF0FE4040F4400070476A
:109F9800FF2313EAD0521EBF13EAD153FF2AFF2B27
:109FA80036D0D21A7F3281EA000C0CF0004C4FF008
:109FB800004343EA002043EA012130B4431A3CBF7E
:109FC80001EB4303013A090AB3FBF1F505FB113331
:109FD8001B02B3FBF1F001FB103300EB05201B0261
:109FE800B3FBF1F505EB00205CEA500050EBC250E2
:109FF80030BC002A09DDFF2A38BF70474FF07F4088
:10A008000CF0004C4CEA500070470CF000407047D0
:10A0180003EAD15393F0FF0F08D192F0FF0F1BD042
:10A028005FEA412C14D04FF440001DE092F0FF0F7E
:10A0380005D14FF07F43B3EB400F10D00CD193F014
:10A04800000F08BF92F0000F06D093F0000F06D063
:10A05800484000F0004070474FF4400004E048409A
:10A0680000F0004040F4000040F0FE40704700BFA0
:10A078004FF4001C1CEB410F98BF1CEB430F11D889
:10A0880051EA030C50EA4C0C5CEA020C0AD004D2E8
:10A0980082428B41804140427047904299418041C1
:08A0A8004042704700207047A0
:10A0B0004FF4001C1CEB410F98BF1CEB430F11D851
:10A0C00051EA030C50EA4C0C5CEA020C0AD004D2B0
:10A0D0009042994180414042704782428B41804189
:08A0E000404270470020704768
:10A0E800C0F3C751D1F19E0108D950F400004FEADE
:10A0F800002020FA01F048BF404270474200B2F108
:10A108007F4F88BF20F0004010F0004058BF6FF02C
:04A11800004070474C
:10A11C0010F0004118BF4042B0FA80F210FA02F37E
:10A12C000DD0D2F19D0241EAC25101EB13205A0627
:10A13C0038BF704700F1010008BF20F001007047E4
:10A14C00C0F3C75191B142004FEA40704FEAD201BF
:10A15C004FEA310101F16051B2F17F4F38BF7047C6
:10A16C0001F1605118BF41F40021704710F000411B
:04A17C000020704708
:04A1800004030904C7
:10A184001803430046006F007200740068002D003D
:08A194004D00490044004900A0
:10A19C00000000000000000001020304060708098B
:10A1AC00537461636B3D0000436F64655468726562
:10A1BC0061643D00456D7074795F000050726F6A88
:10A1CC0065637400206C6F616465642020204155C8
:10A1DC00544F4558453D0000537973436C6F636B86
:10A1EC003D0000002020205465726D696E616C5F2B
:10A1FC0053706C69743D00002020204261756452DC
:10A20C006174653D0000000020204D69646943685D
:10A21C003D0000002870656E64696E6729000000BF
:10A22C002020205350493D004672657131323D006B
:10A23C00487A2050574D313D000000002C50574DAE
:10A24C00323D00002020204672657133343D000001
:10A25C00487A2050574D333D000000002C50574D8C
:10A26C00343D00004D4F54313A0000002020204D69
:10A27C004F54323A000000002020204D4F54333A06
:10A28C0000000000537465703D0000006D73204E9B
:10A29C003D00000044432F50574D00002D2D2D2D17
:10A2AC002D2D2D2D2D2D0000576F726B206F6E20D4
:10A2BC00444D586368616E6E656C3A002846616463
:10A2CC006554696D653D000073204379636C653D91
:10A2DC000000000020426F6F745363656E653D0093
:10A2EC00205761726E696E673A2077696C6C206FCB
:10A2FC0076657272696465204B65726E656C204F71
:10A30C005020772E73616D65206E616D6521200084
:10A31C000000000000000000000000000000000031
:10A32C000000000000000000000000000000000021
:10A33C000000000000000000000000000000000011
:10A34C000000000000000000000000000000000001
:10A35C0000000000000000000000000000000000F1
:10A36C0000000000000000000000000000000000E1
:10A37C0000000000000000000000000000000000D1
:10A38C0000000000000000000000000000000000C1
:10A39C0000000000000000000000000000000000B1
:10A3AC00000000000000000000000100000005009B
:10A3BC000000000000000000000000000000000091
:10A3CC000000000000000000000000000000000081
:10A3DC000000000000000100000004000000040068
:10A3EC000000000000000000000000000000000061
:10A3FC000000010000000000000000000000000050
:10A40C000000000000000000000004000000040038
:10A41C000000040000000400000004000000040020
:10A42C000000000000000000000000000000000020
:10A43C000000000000000000000000000000000010
:10A44C000000000000000000000000000000000000
:10A45C0000000000000000000000000000000000F0
:10A46C0000000000000004000000040000000400D4
:10A47C0000000000000000000000000000000000D0
:10A48C0000000000000004000000000000000500B7
:10A49C00000005000000050000000500000004009D
:10A4AC000000040000000400000000000000010097
:10A4BC00000001000000010000000100000003008A
:10A4CC000000030000000300000003000000030074
:10A4DC000000030000000300000003000000030064
:10A4EC000000030000000300000003000000020055
:10A4FC000000020000000200000002000000020048
:10A50C00000001000000010000000800000008002D
:10A51C00000008000000080000000800000008000F
:10A52C0000000800000008000000080000000800FF
:10A53C0000000800000008000000080000000800EF
:10A54C0000000800000008000000020000000200EB
:10A55C0000000100000001000000010000000100EB
:10A56C0000000100000005000000010000000100D7
:10A57C0000000400000004000000040000000400BF
:10A58C0000000000000000000000000000000000BF
:10A59C0000000000000000000000040000000000AB
:10A5AC00000000000000010000000100000000009D
:08A5BC00000000000000050092
:10A5C4004552524F5200000044524F5000000000C8
:10A5D4004455500000000000535741500000000053
:10A5E4004F56455200000000524F54000000000036
:10A5F4002D524F54000000005049434B000000000E
:10A60400524F4C4C00000000494E4A454354000050
:10A614002B00000000000000312B000000000000AF
:10A624002D00000000000000312D0000000000009B
:10A6340041425300000000005348494654000000C2
:10A64400414E4400000000004F5200000000000092
:10A65400584F5200000000004E4F5400000000000C
:10A664002B2F2D00000000002A0000000000000035
:10A674002F000000000000002A2F0000000000004E
:10A684004D4F4400000000002F4D4F4400000000D7
:10A69400425345540000000042434C520000000065
:10A6A400425453540000000052414E444F4D0000A8
:10A6B4003D3D000000000000213D000000000000BE
:10A6C4003E000000000000003E3D000000000000CD
:10A6D4003C00000000000000553C000000000000A9
:10A6E4003C3D000000000000303D00000000000080
:10A6F400564152434F4E00005245560000000000A0
:10A70400570000000000000052000000000000009C
:10A7140041525241590000004B45593F000000008E
:10A724004B45590000000000454D4954000000000D
:10A734002E000000000000002E4800000000000071
:10A744002E440000000000002E2200000000000043
:10A75400445A0000000000004858000000000000B7
:10A7640052583F0000000000525800000000000052
:10A7740054580000000000004E545800000000002F
:10A784005458220000000000584E4F5000000000B2
:10A794004D5300000000000044530000000000007E
:10A7A400544958000000000054494D450000000081
:10A7B400465245513132000050574D3100000000DF
:10A7C40050574D32000000004652455133340000CA
:10A7D40050574D330000000050574D340000000026
:10A7E4004F480000000000004F4C00000000000033
:10A7F40044414F340000000044414F350000000044
:10A804004950550000000000495044000000000079
:10A81400495A0000000000005244494E0000000064
:10A824005241444300000000494E492D5350490011
:10A834005350490000000000494E492D493243005D
:10A8440049545831000000004954584E000000009B
:10A8540049525831000000004952584E000000008F
:10A8640049414452584E00004D4F543100000000FD
:10A874004D4F5432000000004D4F5433000000008F
:10A88400524547570000000052454752000000005F
:10A89400524547425345540052454742434C5200A7
:10A8A40052454742545354002E5300000000000008
:10A8B40046530000000000004F5053000000000009
:10A8C4005553455200000000534545000000000068
:10A8D4004D454D00000000005354000000000000EE
:10A8E40052554E00000000004E4F2D4442470000D8
:10A8F4004445425547000000464F52474554000026
:10A9040041424F52540000005245504C41434500CF
:10A91400524553544F524500494600000000000080
:10A9240043415345000000003C43415345000000AF
:10A934003E43415345000000454C53450000000090
:10A944005448454E00000000444F00000000000041
:10A95400554E54494C0000005748494C45000000EE
:10A96400414741494E000000464F5200000000009C
:10A974004C4F4F5000000000490000000000000050
:10A98400434F4E5449000000425245414B000000E1
:10A994005A425245414B000052455455524E000014
:10A9A4003A000000000000003B000000000000002E
:10A9B400646F535452000000646F494F5354520063
:10A9C400646F4C4954000000646F56414C55450077
:10A9D400646F524556000000646F49460000000051
:10A9E400646F434153450000646F3C434153450049
:10A9F400646F3E4341534500646F454C534500002A
:10AA0400646F444F00000000646F554E54494C007D
:10AA1400646F5748494C4500646F414741494E00B3
:10AA2400646F464F52000000646F4C4F4F5000005B
:10AA340052502D310000000052502D34000000000F
:10AA44004155544F4558450053504C49540000005B
:10AA540042415544000000004348414E4E454C00DD
:10AA640056494450494400003F00000000000000E3
:10AA740053415645000000004C4F41440000000083
:10AA84005853000000000000585600000000000069
:10AA94005852474200000000584E524742000000FE
:10AAA4005853455400000000584E000000000000B8
:10AAB400583D00000000000058465400000000000B
:10AAC400582B000000000000582D0000000000007A
:10AAD400583000000000000058464C415348000024
:10AAE4005843594300000000582D424F4F54000072
:10AAF400582D534156450000582D4C4F41440000F9
:10AB0400584C2D504152540058520000000000008F
:10AB1400FEE7FEE7FEE7FEE7FEE7FEE7FEE7FEE709
:10AB2400FEE7FEE7FEE7FEE7FEE7FEE7FEE7FEE7F9
:10AB3400FEE7FEE7FEE7FEE7FEE7FEE7FEE7FEE7E9
:10AB4400FEE7FEE7FEE7FEE7FEE7FEE7FEE7FEE7D9
:10AB5400FEE7FEE7FEE7FEE7FEE7FEE7FEE7FEE7C9
:10AB6400FEE7FEE7FEE7FEE7FEE7FEE7FEE7FEE7B9
:10AB7400FEE7FEE7FEE7FEE7FEE7FEE7FEE7FEE7A9
:10AB8400FEE7FEE7FEE7FEE7FEE7FEE7FEE7FEE799
:10AB9400FEE7FEE7FEE7FEE7FEE7FEE7FEE7FEE789
:10ABA400FEE7FEE7FEE7FEE7FEE7FEE7FEE7034813
:10ABB4008546F8F759FB00F003B870470080002081
:10ABC40011488546114C20680434004201D0804766
:10ABD400F9E70F480F49091A082903DB002202602C
:10ABE400043001600C480D49884205D002680430E5
:10ABF40003B4904703BCF7E700208646EC460020E8
:10AC04000021074A9047FEE700800020D0B30008E7
:10AC1400C0770020C07B0020F7AF0008F7AF000822
:04AC2400351A0008D5
:10AC28001EF0040F0CBFEFF30880EFF30980014911
:08AC3800084700002FAF0008DF
:10AC400055534220706C7567676564202E2E2E2048
:10AC50000000000055534220756E706C7567676583
:02AC600064008E
:10AC620010B50446000FF5F790FEC4F30360F5F744
:10AC72008CFEC4F30350F5F788FEC4F30340F5F7E6
:10AC820084FEC4F30330F5F780FEC4F30320F5F726
:10AC92007CFEC4F30310F5F778FE04F00F00F5F71D
:0AACA20074FE2020F5F7EFFC10BD52
:10ACAC001201100102000040830440573D070000D0
:02ACBC00000195
:0EACBE0008B5F6F7A4FD2020F5F7DFFC08BD71
:02ACCC00000086
:10ACCE0010B504462020F5F7D8FC2046F6F797FD80
:02ACDE0010BDA7
:10ACE000120368006F006D0065006D006100640074
:02ACF0006500FD
:0AACF20008B50120FCF7C1F808BD09
:10ACFC001201100100000040830443573D0702017C
:02AD0C00000144
:0AAD0E0008B50020FCF7B3F808BDFB
:10AD1800756E646572666C6F77212000202D2D2D6D
:02AD2800200009
:0EAD2A0008B58920FBF74BFCFDF743FF08BD81
:10AD38004261756452617465206368616E6765730A
:10AD48002074656D706F726172696C792100000002
:10AD58006E65772042617564205261746520736165
:10AD68006D6520666F7220616C6C2050726F6A6529
:10AD78006374732E204E6F74206163746976652046
:10AD88006265666F7265206E657874207379737476
:0AAD9800656D2073746172742E0063
:0EADA20008B58A20FBF70FFCFDF707FF08BD80
:10ADB0002030204348414E4E454C2061636365700E
:10ADC000747320414E59204D494449206368616E97
:10ADD0006E656C20696E20726563656976656420B6
:06ADE0006D736773200093
:0EADE60008B58B20FBF7EDFBFDF7E5FE08BD81
:10ADF4004572726F722300002028636F6C2000007C
:10AE0400206E6F7420666F756E6400005F53796EF8
:10AE140074617820457272005F537461636B2045DE
:10AE2400727200005F436F6D70696C65206F6E6CA9
:10AE3400790000005F4E6F20492F4F436F6D6D20E6
:10AE440041636365737300005F496E76616C696486
:10AE540020436F64652061636365737300000000C1
:10AE64005F6F7574206F6620436F6E74657874002D
:10AE74005F52756E74696D65206F6E6C7920746FA6
:10AE84006B656E005F5468726561642063616E6314
:10AE9400656C6C65640000005F4E756D62657220C0
:10AEA4006F7574206F662052616E67650000000044
:10AEB4005F4469766973696F6E206279205A65729E
:10AEC4006F0000002020636F6D70696C696E6720ED
:06AED400202020202000D8
:0AAEDA0008B50120FEF707FC08BDD3
:06AEE4002849502D3E003C
:0AAEEA0008B50020FEF7FFFB08BDCD
:10AEF40063616E277420534545204B65726E656C03
:10AF0400204F7073000000005573657248656164DA
:10AF140065725F5374727563743D000056617243C9
:0AAF24006F6E3A56616C75653D00D2
:10AF2E004FF0E023D3F82C3D002B00DBFEE74FF073
:10AF3E00E022D2F82C3D43F00043C2F82C3D836949
:06AF4E000233836170472D
:10AF540020636F6E6669726D20772E7570706572EE
:10AF640020636173652027592720000063616E63A5
:06AF7400656C6C656400D1
:10AF7A00844640EA010313F0030F18D18446202ABD
:10AF8A000BD32DE9F007B1E8F807A0E8F807A2F11A
:10AF9A002002202AF7D2BDE8F007042A07D351F885
:10AFAA00043B40F8043BA2F10402042AF7D2002A27
:10AFBA0005D011F8013B00F8013B013AF9D160468E
:02AFCA007047CE
:10AFCC00555342206173207669727475616C20430D
:10AFDC004F4D3D00555342206173204D494449204B
:0BAFEC00696E746572666163653D006C
:10AFF80043466F7274682D444D5820666F72205313
:10B00800544D333247347878204C514650333220EF
:10B01800760000002020286329323032302D323467
:0DB0280020572E536368656D6D65727400CE
:07B038006E6F20555342002A
:10B0400009024300020100803109040000010202EC
:10B050000000052400100105240103000424020758
:10B0600005240600010705830310004009040100C0
:10B07000020A0000000705810240000007050202E5
:03B080004000008D
:07B0840000C20100000008FA
:10B08C000902650002010080310904000000010181
:10B09C00000009240100010900010109040100025A
:10B0AC0001030000072401000141000624020101F4
:10B0BC00000624020202000924030103010201001C
:10B0CC00092403020401010100090581024000006A
:10B0DC0000000525010103090502024000000000E3
:05B0EC00052501010132
:09B0F40028566172436F6E3D00A5
:0DB10000526561642066726F6D20533D0042
:0DB110004B65726E656C3A00444D583A0074
:10B12000313238205352414D2062797465732028A2
:10B13000333220776F72647329207374617274697B
:0BB140006E672066726F6D2030780093
:10B14C00203C2D6E6F742061204B65726E656C20F7
:10B15C004F50206E6F722061206E756D62657200AB
:10B16C00203C2D696E76616C696420666F7220429A
:10B17C0061636B2D4374726C00000000203C2D52F7
:0DB18C00756E74696D65204572726F7200FA
:10B19C0020202841444320696E6974292000000056
:0DB1AC00202028414443206F6666292000C2
:10B1BC002064656275672066696E697368656420D2
:01B1CC000082
:10B1D00020707265736574204261756420526174D9
:10B1E0006520726573746F72656421200000000031
:10B1F000555342205465726D696E616C5F436F6D8B
:10B200002077696C6C20676574206C6F7374210003
:10B210005553415254205465726D696E616C5F43A1
:10B220006F6D2077696C6C20676574206C6F737428
:10B230002100000055534152542077696C6C206303
:10B2400068616E676520746F204D49444920492F1D
:03B250004F21008B
:0FB25400564944203D200000504944203D200031
:05B26400536176650056
:05B26C004C6F6164005D
:10B27400283D456D7074792050726F6A6563742936
:01B2840000C9
:0DB288002050726F6A656374206E6F2E0097
:10B2960010B5044614F8010B28B1F5F7F2F914F8C5
:08B2A600010B0028F9D110BDD5
:10B2AE0010B50446C0F3031303F13000392888BFEC
:10B2BE0003F13700F5F7E1F904F00F0404F1300063
:10B2CE00392888BF04F13700F5F7D7F92020F5F7B4
:04B2DE00D4F910BDD2
:10B2E20010B50446000F1ED1C4F3036014F0706F52
:10B2F2001DD1C4F3035014F4700F1CD1C4F30340E6
:10B3020014F4702F1BD1C4F3033014F4704F1AD10C
:10B31200C4F3032014F4706F19D1C4F3031014F0B2
:10B32200F00F1AD017E0F5F730FBC4F30360F5F71E
:10B332002CFBC4F30350F5F728FBC4F30340F5F7E5
:10B3420024FBC4F30330F5F720FBC4F30320F5F725
:10B352001CFBC4F30310F5F718FB04F00F00F5F71C
:04B3620014FB10BD0B
:10B3660010B504463020F5F78CF97820F5F789F901
:08B376002046FFF7B3FF10BDF4
:10B37E002F2810D9A0F13003DBB2092B09D90A29E5
:10B38E000CD0A0F14103DBB2052B0AD83738C0B27E
:10B39E007047184670474FF0FF3070474FF0FF3040
:08B3AE0070474FF0FF307047BB
:10B3B60038B50546A0F11004207820B1F5F761F9FB
:08B3C6000134A542F8D138BDA5
:10B3D000ADB60008BC02002003750000C3B600082B
:10B3E00000000020F0B30008BC02000000000000D4
:10B3F0000933000819330008413300086D33000891
:10B400008533000899330008BD330008E133000894
:10B41000253400088D340008F53400081135000883
:10B42000213500083D3500084D350008613500081C
:10B43000A9350008C5350008E1350008FD350008CC
:10B440000D360008D90100081D3600085902000811
:10B450005136000889360008BD360008F536000868
:10B4600031370008753700088D370008B1370008FC
:10B47000E5370008093800082D3800085138000861
:10B4800075380008D1370008B9980008A16700088E
:10B4900099380008D538000809390008916D00086E
:10B4A000E94700088547000861480008414800084E
:10B4B000194B0008F3AC0008593900087939000825
:10B4C0001970000805890008314B0008494B000835
:10B4D0000FAD000899390008AD890008D989000826
:10B4E000BD390008DD390008A57300089D72000809
:10B4F000F97300080D7700080576000861770008E9
:10B50000F178000895790008814B0008E94B0008A4
:10B510003D7A0008D97A0008757B00081578000884
:10B520005D7D000825800008698000080D3A00084C
:10B53000FD3A0008B53B0008A93C0008613D000841
:10B54000453E000845840008198600087D8A0008E9
:10B55000B53F0008ED3F00081D400008714000089D
:10B56000C5400008A94800084D420008514C000899
:10B570006D49000849920008214D00086D420008FD
:10B5800079420008854200089D470008A56400082C
:10B5900091420008A995000871960008716800089A
:10B5A00099680008C1680008E96800081169000886
:10B5B000214100084D6900082BAD0008A3AD00082B
:10B5C000E7AD0008756900089D6900085141000851
:10B5D0006D4100089D410008B1410008D9410008B3
:10B5E00001990008E5690008DBAE0008EBAE000831
:10B5F000F143000811440008314400085544000894
:10B6000081440008AD440008D944000805450008FD
:10B61000154500083545000879450008BD45000876
:10B62000D94500081546000895460008A5460008BB
:10B6300075650008459900085956000841570008EB
:10B64000759A0008154E0008F99A0008959B0008A5
:10B65000B54600081958000845580008B5580008B4
:10B660004559000875590008B5590008AD5700083C
:10B67000E14600080947000831470008F58900083D
:10B6800051470008E5570008215A0008A15A000850
:10B690004D5B0008654A0008010000009C5E002028
:0CB6A00020630020246500200024F4003A
:10B6AC00206861680834094204D00022027001301D
:06B6BC000139FBD17047CB
:10B6C20020686168A2680C34124205D00B780370BE
:0AB6D20001300131013AF9D170474F
:040000050800ABB391
:00000001FF
